:020000040000FA
:10000000F0EF2AF08B94000C056ED8CF06F0E95083
:10001000076EEA50086EE150096EE2500A6ED95040
:100020000B6EDA500C6EF350146EF450156EE050F7
:100030000D6E000100500F6E0150106E0250116ED7
:100040000350126E0450136E9DA02AEF00F09EB074
:10005000B2EF1AF00F50006E1050016E1150026E88
:100060001250036E1350046E0D50E06E0D8E07504B
:10007000E96E0850EA6E0950E16E0A50E26E0B50CC
:10008000D96E0C50DA6E1450F36E1550F46E0550A4
:1000900006C0D8FF1000F76AA60FF66E000EF72212
:1000A0000900F550120000018002808080038080EA
:1000B00080808080800480808080808080808080BC
:1000C00080808080800580808080808080808080AB
:1000D0008080808080808080808080808080808020
:1000E000808080808006808080808080808080808A
:1000F0008080808080808080808080808080808000
:1001000080808080808080808080808080808080EF
:1001100080808080808080808080808080808080DF
:100120008080808080078080808080808080808048
:1001300080808080808080808080808080808080BF
:1001400080808080808080808080808080808080AF
:10015000808080808080808080808080808080809F
:10016000808080808080808080808080808080808F
:10017000808080808080808080808080808080807F
:10018000808080808080808080808080808080806F
:10019000808080808080808080808080808080805F
:1001A000808080808008F76AB60FF66E010EF72215
:1001B0000900F550120000010102010202030102D0
:1001C0000203020303040102020302030304020305
:1001D00003040304040501020203020303040203EF
:1001E00003040304040502030304030404050304D5
:1001F00004050405050601020203020303040203C9
:1002000003040304040502030304030404050304B4
:10021000040504050506020303040304040503049E
:100220000405040505060304040504050506040584
:100230000506050606070102020302030304020382
:100240000304030404050203030403040405030474
:10025000040504050506020303040304040503045E
:100260000405040505060304040504050506040544
:100270000506050606070203030403040405030438
:100280000405040505060304040504050506040524
:10029000050605060607030404050405050604050E
:1002A00005060506060704050506050606070506F4
:1002B000060706070708F76AC60FF66E020EF72252
:1002C0000900F55012000002080A2022282A808224
:1002D000888AA0A2A8AAF76AE60FF66E020EF72295
:1002E0000900F55012000102050B162C58B1F76AEF
:1002F000FE0FF66E020EF7220900F5501200806420
:1003000040170B060202ECCFFAFFED52EFCFF9FFD8
:10031000000C246A286A2EA602D0010E246E2FA893
:1003200002D0010E241A2FAC02D0010E286E2FAE7F
:1003300002D0010E281A2850241A286A2EAE02D0A4
:10034000010E286ED8902E36D8902F36282C01D04A
:100350002F802452D8A42E80246A47AE02D0010EEA
:10036000246E47AA02D0010E241A47A802D0010E1B
:10037000241A47A402D0010E241AD89047362450DC
:100380004712BDEF1AF047B003D0800E016E25D0A2
:1003900047B203D0C00E016E20D047B403D0E00EA8
:1003A000016E1BD047B603D0F00E016E16D047B8D1
:1003B00003D0F80E016E11D047BA03D0FC0E016EC7
:1003C0000CD047BC03D0FE0E016E07D047BE03D051
:1003D000FF0E016E02D0FF0E016EBFEF1AF078CA59
:1003E00031F0246A79CA20F031521CE03150CF5CE0
:1003F00003E3000E016EC2D19EA003D0000E016E79
:10040000BDD1CF50315C2A0803E2FF0E2D6E09D01A
:10041000CF50315C006ED89000342D6E2D502D24BD
:100420002D2609D09EA007D09E902006205203E1E1
:10043000000E016EA3D19E929EA2FED7CCCF22F0D9
:1004400022A001D002D00000000022A201D003D0DF
:1004500000000000000022A401D005D00000000030
:1004600000000000000000006B9A6B986B88A4BA33
:100470006E50A4BA6E50A4AAFED76E50016E01C091
:1004800023F02D2E01D0B0D7233C01D001D0F3D7DB
:10049000A4AAFED76ECF23F02D2E01D0A5D72350CE
:1004A000FADD016E01C022F02250070807E322C0E6
:1004B00029F0080ED8802254246E04D022AE01D038
:1004C00093D7E6D7A4AAFED76ECF23F02D2E01D066
:1004D0008BD72350FF0ADFDD016E01C022F02250CE
:1004E00007080BE3225024242A6E120E2A5C0C0803
:1004F00001E27AD7080E242606D0080E242622AE62
:1005000001D072D7DFD7A4AAFED76ECF23F02D2E4D
:1005100001D06AD72350BFDD016E01C022F0225006
:1005200007080BE3225024242B6E2F0E2B5C0208AD
:1005300001E25AD7080E242606D0080E242622AE41
:1005400001D052D7E0D7A4AAFED76ECF23F02D2E2C
:1005500001D04AD72350FF0A9EDD016E01C022F070
:10056000225007080AE3225024242C6E2A502C5CC7
:10057000D10F020801E238D706D0080E242622AE99
:1005800001D032D7E0D72A502A242B242B24A00FC5
:10059000286E2C502824D00F286E030E28262830D1
:1005A000226E22323F0E22162838246E0F0E241699
:1005B0002838206E20322032030E20162D6A28BEE5
:1005C0002D802450222420242D24006ED890003029
:1005D000286E0C0E285E29502826070E28162A5051
:1005E0002B5CD8802A54266E285226E09E929E923A
:1005F0009EA2FED7CCCF22F022A001D002D00000D4
:10060000000022A201D003D000000000000022A4BC
:1006100001D005D000000000000000000000000034
:10062000050E006E002EFED7000000000000000046
:10063000282EFCD7CC6A9E929E929EA2FED7CCCF4B
:1006400022F022A001D002D00000000022A201D09E
:1006500003D000000000000022A401D005D000005B
:10066000000000000000000000006B9A6B986B888F
:10067000A4BA6E50A4BA6E50280E2D6E010E226ED2
:1006800022520AE0A4AAFED76E50016E01C022F0E9
:100690002D2E01D072D0F4D722520AE1A4AAFED79F
:1006A0006E50016E01C022F02D2E01D066D0F4D71D
:1006B0002250F0080AE12650040806E2A4AAFED758
:1006C0006E50016E01C022F008D022B806D0A4AA54
:1006D000FED76E50016E01C022F0286AA4AAFED790
:1006E0006E50016E01C022F02D2E01D046D0223C6A
:1006F00004D0D8902836288007D0225204E1D89020
:100700002836289001D070D63F0E2816285032087F
:1007100001E113D0A4AAFED76E50016E01C022F0F1
:100720002D2E01D02AD0A4AAFED76E50016E01C092
:1007300022F02D2E01D021D0D1D79E929EA2FED79D
:10074000CCCF22F022A001D002D00000000022A2D3
:1007500001D003D000000000000022A401D005D089
:100760000000000000000000000000000A0ECF6E34
:10077000220ECE6E010E016E01D036D6000CCF5087
:10078000000803E2000E016E7BD0010E0A017A6FB1
:100790007ACA31F09E903150FD0802E2FD0E316EB2
:1007A0003150CF5CFDE3CEA6FED7CECF22F022A003
:1007B00001D002D00000000022A201D003D000002E
:1007C0000000000022A401D005D0000000000000BD
:1007D000000000000000CC6A9E929EA2FED7CCCF03
:1007E00022F022A001D002D00000000022A201D0FD
:1007F00003D000000000000022A401D005D00000BA
:1008000000000000000000000000E30E326EC9503E
:10081000206E3250C96EC7A0FED78E0E326EC95000
:10082000206E3250C96EC7A0FED7380E326EC95046
:10083000206E3250C96EC7A0FED7E30E326EC9508B
:10084000206E3250C96EC7A0FED78F0E326EC950CF
:10085000206E3250C96EC7A0FED7C00E326EC9508E
:10086000206E3250C96EC7A0FED7E00E326EC9505E
:10087000206E3250C96EC7A0FED7010E016E000176
:10088000000C1C2C36D045502E1445240A01776FDD
:10089000786B77CA79FA0001A2DD015203E0010EFC
:1008A000016E39D0CF6ACE6A979A8E9A98988F88BF
:1008B00066DF979A8E8A98988F888C820A01786B67
:1008C000020E796F00018BDD015203E0010E016E13
:1008D00022D02EC078FA010E0A01796F00017FDD67
:1008E000015203E0010E016E16D0000E016E13D00E
:1008F00012D045502E1445240A01776F786B77CAC1
:1009000079FA00016CDD015203E0010E016E03D0A3
:10091000000E016E00D0EAEF1AF01F50F00B006ECF
:10092000003A0F0E00160050036AC5DC016E01C0CC
:100930002AF01F500F0B036ABEDC016E01C029F0C4
:10094000246A0A01775362E1979A8E9A98988F8861
:10095000CF500A0803E2000E016ED6D00B0E7A6F5C
:100960007ACA31F09E903150FD0802E2FD0E316EE0
:100970003150CF5CFDE3CEA6FED7CECF22F022A031
:1009800001D002D00000000022A201D003D000005C
:100990000000000022A401D005D0000000000000EB
:1009A000000000000000CC6A9E929EA2FED7CCCF31
:1009B00022F022A001D002D00000000022A201D02B
:1009C00003D000000000000022A401D005D00000E8
:1009D000000000000000000000002AC032F0C950F2
:1009E000206E3250C96EC7A0FED729C032F0C95060
:1009F000206E3250C96EC7A0FED7979A8E8A9898FB
:100A00008F888C82000E016E7FD07ED0979A8E8A5E
:100A100098988F888C92CF500A0803E2000E016EDE
:100A200073D00B0E7A6F7ACA31F09E903150FD0868
:100A300002E2FD0E316E3150CF5CFDE3CEA6FED753
:100A4000CECF22F022A001D002D00000000022A2CE
:100A500001D003D000000000000022A401D005D086
:100A6000000000000000000000000000CC6A9E9220
:100A70009EA2FED7CCCF22F022A001D002D000004F
:100A8000000022A201D003D000000000000022A438
:100A900001D005D0000000000000000000000000B0
:100AA0006B9A6B986B88A4BA6E50A4BA6E50286A81
:100AB0002850070821E3A4AAFED76E50016E01C09A
:100AC00022F022500001D3EC00F0016E01C02BF0A7
:100AD000A4AAFED76E50016E01C022F02250D3ECC2
:100AE00000F0016E2B26D89024322B500108D8A09C
:100AF000248E282A0A01DCD7979A8E8A98988F88A4
:100B00008C822450016E00D00001000C0A01C051FB
:100B1000C203F3CF01F0F4CF00F0C303F35000267B
:100B2000C151C203F3500020026E0001000C979ADD
:100B30008E8A98988F888C928B9AC69A8B9ACF506F
:100B40000E0804E2C68A000E016EB8D00F0E0A012C
:100B50007A6F7ACA31F09E903150FD0802E2FD0EA4
:100B6000316E3150CF5CFDE3CEA6FED7CECF22F062
:100B700022A001D002D00000000022A201D003D0A8
:100B800000000000000022A401D005D000000000F9
:100B90000000000000000000CC6A9E929EA2FED7DA
:100BA000CCCF22F022A001D002D00000000022A26F
:100BB00001D003D000000000000022A401D005D025
:100BC0000000000000000000000000006B9A6B981D
:100BD0006B88A4BA6E50A4BA6E50226A246A773722
:100BE0007837773778377737783777377837773791
:100BF000783777377837C00E7717A4AAFED76E50AC
:100C0000016E286A28500A083FE378AF06D0979A09
:100C10008E9A98988F888B8A06D0979A8E8A989801
:100C20008F888C928B9A22500001D3EC00F0016ED9
:100C300024262450070804E228060A0125D00001D2
:100C4000A4AAFED76E50016E01C022F0A4AAFED75E
:100C50006E50016E01C022F0A4AAFED76E50016E44
:100C600001C022F02250D3EC00F0016E01C024F04C
:100C7000A4AAFED76E50016E01C022F0D8900A01DE
:100C800077377837282ABED78B9AC68A979A8E8A62
:100C900098988F888C8228500B0805E1010E016E10
:100CA00000010CD00A012850090805E3020E016E6C
:100CB000000104D00A01000E016E0001000CC68A7A
:100CC000979A8E9A98988F88180E0A017A6F7ACA26
:100CD00031F09E903150FD0802E2FD0E316E315030
:100CE000CF5CFDE3CEA6FED7CECF22F022A001D06E
:100CF00002D00000000022A201D003D000000000BA
:100D0000000022A401D005D0000000000000000077
:100D100000000000CC6A9E929EA2FED7CCCF22F0AB
:100D200022A001D002D00000000022A201D003D0F6
:100D300000000000000022A401D005D00000000047
:100D40000000000000000000AA0E326EC950206EA4
:100D50003250C96ECA0E326EC7A0FED7C950206E7F
:100D60003250C96E2EA403D0170E326E02D0740E0C
:100D7000326EC7A0FED7C950206E3250C96E32C045
:100D800029F00C0E5324020F326EC7A0FED7C950B3
:100D9000206E3250C96E246A245007080BE32A6A79
:100DA00029B62A2A29BC2A2AD89029362AB029808D
:100DB000242AF2D7295000019719326EC7A0FED716
:100DC000C950206E3250C96E246A245007080BE3C4
:100DD0002A6A29B62A2A29BC2A2AD89029362AB072
:100DE0002980242AF2D729509819326EC7A0FED73D
:100DF000C950206E3250C96E246A245007080BE394
:100E00002A6A29B62A2A29BC2A2AD89029362AB041
:100E10002980242AF2D72950AA0A326EC7A0FED709
:100E2000C950206E3250C96E246A245007080BE363
:100E30002A6A29B62A2A29BC2A2AD89029362AB011
:100E40002980242AF2D72950AA0A326EC7A0FED7D9
:100E5000C950206E3250C96E246A245007080BE333
:100E60002A6A29B62A2A29BC2A2AD89029362AB0E1
:100E70002980242AF2D72950AA0A326EC7A0FED7A9
:100E8000C950206E3250C96E246A245007080BE303
:100E90002A6A29B62A2A29BC2A2AD89029362AB0B1
:100EA0002980242AF2D72950AA0A326EC7A0FED779
:100EB000C950206E3250C96E286A28500B0821E3B1
:100EC000246A245007080BE32A6A29B62A2A29BC77
:100ED0002A2AD89029362AB02980242AF2D7036AF0
:100EE0002850230FE96E010E0320EA6EEF502918F7
:100EF000326EC7A0FED7C950206E3250C96E282A64
:100F0000DCD753C02DF0286A2D50285C21E2246ADA
:100F1000245007080BE32A6A29B62A2A29BC2A2A60
:100F2000D89029362AB02980242AF2D7036A28507B
:100F3000970FE96E000E0320EA6EEF502918326E0B
:100F4000C7A0FED7C950206E3250C96E282ADCD700
:100F5000246A245007080BE32A6A29B62A2A29BCE6
:100F60002A2AD89029362AB02980242AF2D7295053
:100F700001013D19326EC7A0FED7C950206E325014
:100F8000C96E246A245007080BE32A6A29B62A2A64
:100F900029BC2A2AD89029362AB02980242AF2D7B7
:100FA00029503E19326EC7A0FED7C950206E32506C
:100FB000C96E326AC7A0FED7C950206E3250C96EC2
:100FC000C7A0FED71A8A010E016E0001E1EF1BF0E7
:100FD0001AAC04D01A9C1A90536A03D01A821A9041
:100FE000536A000E016EEEEF1BF0206AA4AAFED732
:100FF0006E50016E01C022F02250E709FF0803E1A4
:10100000010E226E01D0226A22B0208EA4AAFED741
:101010006E50016E01C022F02250E709FF0803E183
:10102000010E226E01D0226A22B0208CA4AAFED723
:101030006E50016E01C022F02250E709FF0803E163
:10104000010E226E01D0226A22B0208AA4AAFED705
:101050006E50016E01C022F02250E709FF0803E143
:10106000010E226E01D0226A22B02088A4AAFED7E7
:101070006E50016E01C022F02250E709FF0803E123
:10108000010E226E01D0226A22B02086A4AAFED7C9
:101090006E50016E01C022F02250E709FF0803E103
:1010A000010E226E01D0226A22B02084A4AAFED7AB
:1010B0006E50016E01C022F02250E709FF0803E1E3
:1010C000010E226E01D0226A22B02082A4AAFED78D
:1010D0006E50016E01C022F02250E709FF0803E1C3
:1010E000010E226E01D0226A22B02080000C206AFC
:1010F000A4AAFED76E50016E01C022F02A6A29B65A
:101100002A2A29BC2A2AD89029362AB02980225096
:10111000E709FF0803E1010E226E01D0226A29507F
:10112000221A22B0208EA4AAFED76E50016E01C0F2
:1011300022F02A6A29B62A2A29BC2A2AD8902936D6
:101140002AB029802250E709FF0803E1010E226E30
:1011500001D0226A2950221A22B0208CA4AAFED7DC
:101160006E50016E01C022F02A6A29B62A2A29BCD3
:101170002A2AD89029362AB029802250E709FF0868
:1011800003E1010E226E01D0226A2950221A22B0F8
:10119000208AA4AAFED76E50016E01C022F02A6AEE
:1011A00029B62A2A29BC2A2AD89029362AB0298089
:1011B0002250E709FF0803E1010E226E01D0226AE6
:1011C0002950221A22B02088A4AAFED76E50016EA0
:1011D00001C022F02A6A29B62A2A29BC2A2AD890D4
:1011E00029362AB029802250E709FF0803E1010EC1
:1011F000226E01D0226A2950221A22B02086A4AA87
:10120000FED76E50016E01C022F02A6A29B62A2A42
:1012100029BC2A2AD89029362AB029802250E709E9
:10122000FF0803E1010E226E01D0226A2950221A22
:1012300022B02084A4AAFED76E50016E01C022F015
:101240002A6A29B62A2A29BC2A2AD89029362AB0FD
:1012500029802250E709FF0803E1010E226E01D028
:10126000226A2950221A22B02082A4AAFED76E50E8
:10127000016E01C022F02A6A29B62A2A29BC2A2A2C
:10128000D89029362AB029802250E709FF0803E1C7
:10129000010E226E01D0226A2950221A22B020802B
:1012A000000C286A285007084EE3A4AAFED76E5007
:1012B000016E2A6A29B62A2A29BC2A2AD8902936F8
:1012C0002AB02980D89028340A017B6B7A6F830E6C
:1012D0007A25E96E010E7B21EA6EEF502B5C23E14B
:1012E000A4AAFED76E50016E2A6A29B62A2A29BC02
:1012F0002A2AD89029362AB02980D89028347B6BA6
:101300007A6F010E7A25016E000E7B21036E01506B
:10131000830FE96E010E0320EA6EEF502C5C02E1B0
:10132000010E246E0DD0A4AAFED76E50016E2A6A5B
:1013300029B62A2A29BC2A2AD89029362AB02980F7
:10134000282A0001AFD7286A28500F080FE3A4AA63
:10135000FED76E50016E2A6A29B62A2A29BC2A2A8B
:10136000D89029362AB02980282AEED77BEF13F0AF
:101370000A01BD6BBC6BBE6BBE510B082EE3BDCA30
:10138000BFFABCCABDFABFCABCFA036ABE51B725D0
:10139000E96EB8510320EA6EEF50BD1BBD39006EF7
:1013A0000F0E00160050BD1BBD39006EF00E00166A
:1013B0000050BC1BBD31006E003200321F0E001603
:1013C0000050BC1BBD39006EF00E00160050D890C6
:1013D00000360050BD1BBE2BCFD7BE6BBB51BE5DD0
:1013E0002EE2BDCABFFABCCABDFABFCABCFA036AC4
:1013F000BE51B925E96EBA510320EA6EEF50BD1B0C
:10140000BD39006E0F0E00160050BD1BBD39006EB9
:10141000F00E00160050BC1BBD31006E00320032D1
:101420001F0E00160050BC1BBD39006EF00E0016DA
:101430000050D89000360050BD1BBE2BCFD7C16BDB
:10144000BCCAC0FA010EC36FC26B000186EC05F086
:1014500002C0C1FA01C0C0FA0A01BD510124016EE7
:10146000000E0220036E0350026E0001000C1AA051
:1014700003D0010E016E02D0000E016E000CF7DFEA
:10148000015208E01AAC03D01A9C1A9002D01A92AA
:101490001A90536A52EF0AF018980101936B826B0D
:1014A0000001EDD7000C0A01B65302E1010EB66F40
:1014B0001ABE03D0000E016E25D01AA003D0000E74
:1014C000016E20D053C024F144C025F154C02EF148
:1014D000010EB86F230EB76FBA6B970EB96F53C07A
:1014E000BBFA000145DF02C056F001C055F056C0FE
:1014F0003DF155C03EF1B6CA52F0542A1A80010E91
:10150000016E0A010001000CB2DF015201E0C4DFEC
:10151000B70E976F800E986F996B030E0A017E6F5E
:101520000101FA533CE00A017E517E2B036A970FBA
:10153000E96E000E0320EA6EEA0EEF6E7E517E2BFE
:10154000036A970FE96E000E0320EA6E800EEF6EBD
:101550007E517E2B036A970FE96E000E0320EA6E20
:10156000EF6A7E517E2B036A970FE96E000E03200F
:10157000EA6EF00EEF6E7E517E2B036A970FE96ED6
:10158000000E0320EA6EC00EEF6E7E517E2B036AC2
:10159000970FE96E000E0320EA6EEF6A0101FB531C
:1015A0001EE00A017E517E2B036A970FE96E000E42
:1015B0000320EA6EF70EEF6E7E517E2B036A970FC3
:1015C000E96E000E0320EA6EEF6A7E517E2B036AFD
:1015D000970FE96E000E0320EA6EEF6A0101F853DF
:1015E0001FE00A017E517E2B036A970FE96E000E01
:1015F0000320EA6ED60EEF6E7E517E2B036A970FA4
:10160000E96E000E0320EA6ED00EEF6E7E517E2B47
:10161000036A970FE96E000E0320EA6EEF6A01017C
:10162000FD531FE00A017E517E2B036A970FE96E7E
:10163000000E0320EA6E8D0EEF6E7E517E2B036A44
:10164000970FE96E000E0320EA6E880EEF6E7E5152
:101650007E2B036A970FE96E000E0320EA6EEF6A95
:101660000101F9531FE00A017E517E2B036A970F97
:10167000E96E000E0320EA6E750EEF6E7E517E2B32
:10168000036A970FE96E000E0320EA6EC80EEF6E34
:101690007E517E2B036A970FE96E000E0320EA6EDF
:1016A000EF6A0101FE531FE00A017E517E2B036A9F
:1016B000970FE96E000E0320EA6E670EEF6E7E5103
:1016C0007E2B036A970FE96E000E0320EA6E180E58
:1016D000EF6E7E517E2B036A970FE96E000E03209A
:1016E000EA6EEF6A0101FC531FE00A017E517E2B76
:1016F000036A970FE96E000E0320EA6E690EEF6E23
:101700007E517E2B036A970FE96E000E0320EA6E6E
:10171000980EEF6E7E517E2B036A970FE96E000ED6
:101720000320EA6EEF6A01017ECA53F01E0E0A0121
:10173000B66F0001B8DE015201E01A8C000E016E96
:10174000000C0A01C751E96EC8CAEAFFEF50CA6F20
:10175000C551E96EC6CAEAFFEF50C96FCB6BC451E1
:10176000CB5D2EE2CACACCFAC9CACAFACCCAC9FA37
:10177000036ACB51C225E96EC3510320EA6EEF50D4
:10178000CA1BCA39006E0F0E00160050CA1BCA3998
:10179000006EF00E00160050C91BCA31006E0032F8
:1017A00000321F0E00160050C91BCA39006EF00E21
:1017B00000160050D89000360050CA1BCB2BCFD754
:1017C000C551E96EC6CAEAFFC9CAEFFFC751E96E43
:1017D000C8CAEAFFCACAEFFF0001000C0A01C451DF
:1017E000016AC35D03E2C351006E0CD0006A080EAB
:1017F000C56FC3370036C451005CD8B0006E0136E7
:10180000C52FF7D70001000C958C9586959E8C8E80
:10181000000CFADF000C958C0000958600008C9C73
:10182000959C00008C969596000C080E016E0000A9
:1018300000008C96959600000A01CC378C9CD8B09D
:10184000958CD8A0959C958683A6FED7012E01D0B5
:1018500002D00001ECD700008C9695960000958C84
:1018600000000000958683A6FED7016A000083BCB5
:1018700001808C9695968C9C959C0001000CCBCA9F
:10188000CCFAD3DF0150000C959C0000958683A60E
:10189000FED70000000000000000958C0000000C46
:1018A000BADFA00E0A01CB6F0001E9DF015204E1AB
:1018B000EBDF010E016E02D0000E016E000C0A017A
:1018C000CA51C00BCC6FCB51CD6FCC51CA5D006EED
:1018D000CD51CB59036E0050FF0A410F016E00013C
:1018E000000C0A01C96BC86BC3CACBFAC2CACAFAD8
:1018F0000001E5DF0A01C75303E1C651015C03E2C1
:10190000010E016E59D0000186DFA00E0A01CB6FD7
:101910000001B5DF015206E0B7DF020E016E0A01D9
:101920004BD000010A0EE8CFEAFFC30EE96EEFCFFD
:10193000CAFACACACBFAA3DF015206E0A5DF040E39
:10194000016E0A0139D000010A0EE8CFEAFFC20E8B
:10195000E96EEFCFCAFACACACBFA91DF015206E0AC
:1019600093DF080E016E0A0127D000010A01C95158
:10197000C75D1DE303E1C651C85D19E2C451C82526
:10198000E96EC551C921EA6EEFCFCAFACACACBFACD
:10199000000175DF015205E077DF100E016E0A01CC
:1019A0000BD00A01C82BD8B4C92B0001DFD7000126
:1019B0006BDF000E016E0A010001000C2CDFA00E8F
:1019C0000A01CB6F00015BDF015204E05DDF010E15
:1019D000016E2CD00A0EE8CFEAFFC20EE96EEFCFFF
:1019E000C4FAC4CACBFA4BDF015204E04DDF020E49
:1019F000016E1CD00A0EE8CFEAFFC10EE96EEFCFF0
:101A0000C4FAC4CACBFA3BDF015204E03DDF020E48
:101A1000016E0CD0C3CACBFA32DF015204E034DFCE
:101A2000030E016E03D030DF000E016E4EEF0EF09C
:101A30000A017F6BDCC07EFA0A0EEA6E810EE96E47
:101A4000E26ADD0EE16E280E016EE6CFEEFF012E9A
:101A5000FCD781CA80FA8053D8A48CD082CAF3F90B
:101A600083CAF4F984CAEFF985CAF0F90901F16B68
:101A7000F26B050E0A017E5DC16F0A0EC36F860E02
:101A8000C26FC1CAC4FA090EC66FF10EC56F090E46
:101A9000C86FF20EC76F000154DE010E0901F56F29
:101AA000020107250A01C26FC2CAC3FA08C2C4FAFA
:101AB000000194DED89000360050036AFF0FE96EF3
:101AC000010E0320EA6EECCF03F0ED52EF50090156
:101AD000ED6F03C0EEF900019CDE0A017F6B00018F
:101AE000DFDE015203E10A01FAD70001EEC9C3FAB1
:101AF000EDC9C2FA0A0E0A01C56F820EC46FC76B28
:101B0000040EC66F0001EDDE01C07FFA200E090150
:101B1000ED27000EEE230001C3DE015203E10901AF
:101B2000FAD70001050E0A017E5DC16FEEC9C3FA46
:101B3000EDC9C2FA0A0EC56F860EC46FC76BC1CA63
:101B4000C6FA0001CEDE01500A017F137E51090161
:101B5000ED250A01C16F000E0901EE210A01C26FD5
:101B6000050EC15D0901ED6F000E0A01C2590901A0
:101B7000EE6F43D00901F5510A01805D3FE1010E8E
:101B80007E5DC16F0A0EC36F820EC26FC1CAC4FAF6
:101B9000090EC66FF10EC56F090EC86FF20EC76F42
:101BA0000001CFDD0901F52B000133DE010E0A0132
:101BB0007E5DC16FEEC9C3FAEDC9C2FA0A0EC56FE8
:101BC000820EC46FC76BC1CAC6FA00018ADE01501B
:101BD0000A017F137E510901ED250A01C16F000E34
:101BE0000901EE210A01C26F010EC15D0901ED6F0D
:101BF000000E0A01C2590901EE6F0A01010E090126
:101C0000F35D0A01805D53E1010E0901F55D0A01F2
:101C1000805D4DE1090EC36FEF0EC26F010EC46F00
:101C2000090EC66FF10EC56F090EC86FF20EC76FB1
:101C3000000187DD090E0A01C36FF00EC26F010EAD
:101C4000C46F090EC66FF10EC56F090EC86FF20E94
:101C5000C76F000176DD0901F15324E1F25322E15F
:101C60000A017F53D8B402D009011CD00101948D20
:101C7000010E020107250A01C26FC2CAC3FA08C2D7
:101C8000C4FA0001ABDD00C007F2C3DD300E0A016B
:101C9000C26FC16B07C2C3FA000190D601500A019E
:101CA0007F130901F16BF26BF36BF56B0A017F5146
:101CB000016E0001000C000E18B8010E010803E1CE
:101CC000020E016E31D0400ED8800101825502080B
:101CD00006E3010E016E000127D026D00101036A40
:101CE0008251420FE96E010E0320EA6E7FCAEFFFB8
:101CF000010E8225036A420FE96E010E0320EA6E8F
:101D000080CAEFFF020E8225036A420FE96E010EC0
:101D10000320EA6EEF6A020E8225936F030E82277C
:101D2000000E016E000100D0000C000E18B8010E6C
:101D3000010803E1020E016E23D0400ED88001019C
:101D40008255000A06E1010E016E000119D018D07B
:101D50000101036A9351420FE96E010E0320EA6EFE
:101D6000EF2A036A8251420FE96E010E0320EA6EE8
:101D70007FCAEFFF010E8227000E016E000100D026
:101D8000000C1ABE03D0000E016E25D01AA003D09D
:101D9000000E016E20D0EA6A970EE96E010EE26E27
:101DA000420EE16E400E016EE6CFEEFF012EFCD733
:101DB00082C153F07FCAB6FA53EC0AF0015208E030
:101DC0000101826B936B010E016E000104D003D000
:101DD000000E016E00D0000C0A017E6BDDC07EFAA1
:101DE000020108510A017E5D05E27ECA07F2010187
:101DF000948D0A01600E7F6F780E806F00015BDFAB
:101E000007C27FFA92DF7ECA7FFA8FDF140E0A01C3
:101E10007F6F0001B6DF02010751016E0001000C67
:101E20000A017C6B7D6BD8907B35036A330FE96EBA
:101E3000000E0320EA6EECCF03F0ED52EF507C6F02
:101E400003C07DFA7C5302E17D530BE00A0EEA6E7B
:101E50007C0EE96E000183EC01F0015006D005D044
:101E60000A01FF0E016E000100D0000C0A01B96BDF
:101E7000BA6BBA51070818E3BA51B825036AB625F8
:101E8000E96EB7510320EA6EEFCFBCFA030EBA2514
:101E9000036A230FE96E010E0320EA6EEF50BC5D6A
:101EA000D8B4B92BBA2BE5D7B951080803E1010E14
:101EB000016E1AD0B96BBA6BBA5107080DE3BA516B
:101EC000B825036AB625E96EB7510320EA6EEF3CE8
:101ED00001D0B92BBA2BF0D7B951080803E1010E94
:101EE000016E02D0000E016E0001000C7BCA1DF0D5
:101EF000000C7BCA45F054EF12F0979C8E9C000CAE
:101F00009D901A9E1AA003D01A901A921A9C02EC65
:101F100000F0F3DF8C8498968F96000C0101966B8D
:101F2000956B986B976B9A6B996B9C6B9B6B9E6B8D
:101F30009D6BA76BA66BC00EA56FA46B9F6BA06B70
:101F4000A16B9493A26BA36B94950001000CFF0E00
:101F5000D880CF540A01BB6BBA6FBBCAC1FABACAE8
:101F6000C0FAC36B330EC26F000186EC05F002C0ED
:101F7000B9FA01C0B8FA0A01B851016EB951026E3E
:101F80000001E8EF0FF0016A026A006A036A0A01C1
:101F9000BD5102E1BC5118E0100EBE6FD890BA37A7
:101FA000BB3700360336BD51035C02E1BC51005C17
:101FB00007E3BC51005ED8A00306BD51035ED88084
:101FC00001360236BE2FEAD700000001000CBFD751
:101FD00002C0B7FA01C0B6FAC80E0A01B65DB86F02
:101FE000000EB759B96FB9CABBFAB8CABAFABD6B15
:101FF000320EBC6F0001C7DF0150000CF250036EBF
:10200000F29EA69CA68EA6840F01550EA76EAA0E60
:10201000A76EA68200000350F2120001000C0A0114
:10202000B56B0A0EEA6E7B0EE96EE26ADD0EE16EBA
:102030003A0E016EE6CFEEFF012EFCD70A0EB76F07
:102040007B0EB66FB86B000111DF0152D8B470D1AE
:102050000A018353D8A4ADD08453D8A4AAD00101D7
:102060009953D8B402D00A01A4D09A53D8B402D05C
:102070000A019FD0010EE8CFEAFF980EE96E8CCAE4
:10208000EFFF010EE8CFEAFF970EE96E8DCAEFFF72
:1020900098510B0807E303E19751940803E3010EFD
:1020A0000A01B56F0A01852D60D0865142085DE1B5
:1020B000875114085AE1B55358E000012FDF010E93
:1020C000E8CFEAFF960EE96E88CAEFFF010EE8CF6F
:1020D000EAFF950EE96E89CAEFFF8ACAA2F18BCAA0
:1020E000A3F109EC0CF073DF015025083CE29EC11E
:1020F000C3FA9DC1C2FA0A0E0A01C56F8A0EC46FE7
:10210000C76B250EC66F000171EC0CF001522BE17C
:10211000400E01019D27000E9E239C6B010E9B6FBC
:102120009A6B020E996F000137EC0AF0015202E03F
:102130004CEC0AF0A50E976F0E0E986F996BC60EB9
:102140009A6F580E9B6F020E9C6F9D6B010E9E6FD7
:10215000080E536E1E0E0A01B66F000153EC0AF012
:10216000015201E01A8C23D00A01A50E0001976FDD
:102170000E0E986F996BC60E9A6F580E9B6F060ED7
:102180009C6FFF0E9D6F9E6F010E9F6F420EA06FA2
:10219000140EA16FB5CAA2F00C0E536E1E0E0A01EA
:1021A000B66F000153EC0AF0015201E01A8CC0D066
:1021B0000A01010EE8CFEAFF9A0EE96EEF50835D47
:1021C000D8A4B5D0010EE8CFEAFF990EE96EEF5022
:1021D000845DD8A4ACD001019E51790828E303E1C5
:1021E0009D51600824E3000109EC0CF0F0DE015081
:1021F00020081BE29EC1C3FA9DC1C2FA0A0E0A0161
:10220000C56F850EC46FC76B200EC66F000171ECE1
:102210000CF001520AE1200E01019D27000E9E23C1
:102220009AC19CF199C19BF1000147D00101D08C6A
:10223000A6C1F8FFA5C1F7FFA4C1F6FFF650070B32
:10224000006EF80EF6160A000A0EEA6E850EE96EAA
:10225000200EE8CF01F00050022602040709026EAA
:10226000022AF650006609D0010F3F0B06E1A6884E
:1022700009000001C3DE0A000101006607D0EECFAD
:10228000F5FF015204E00F00010603D000060B0029
:102290000C00070EF614070A03E10001AFDE01018E
:1022A000022EDFD7F86A200EA427000EA523A6234E
:1022B000A7239AC19CF199C19BF101019C51965DA4
:1022C00030E303E195519B5D2CE2000137EC0AF00D
:1022D000015202E04CEC0AF0A50E976F0E0E986FBB
:1022E000996BC60E9A6F580E9B6F020E9C6F010E73
:1022F000E8CFEAFF9A0EE96EEF509D6F010EE8CF2E
:10230000EAFF990EE96EEF509E6F080E536E1E0E97
:102310000A01B66F000153EC0AF0015201E01A8C79
:102320000101020E9927000E9A23A06B9F6B0001FA
:1023300001019485000166EF12F0A69CA1987ECA67
:10234000A9FF7FCAA8FFA69EA684550EA76EAA0E57
:10235000A76EA682A1A8FED7A694A198000CA69C61
:102360007FCAA9FFA69EA680A850016E000C0A0194
:102370007B6B7B51070829E3060E7B25036AD70F89
:10238000E96E000E0320EA6EEFCF7DFA7BCA7EFA7B
:102390007DCA7FFA0001D1DF030E0A017B25036AA3
:1023A000230F016E010E032201507D6F03C07EFAE0
:1023B0007BCA7FFA0001D3DF7ECAEAFF7DCAE9FF4C
:1023C00001C0EFFF0A017B2BD4D7000137EC0AF0E4
:1023D000015202E04CEC0AF0A50E976F0E0E986FBA
:1023E000996B6D0E9A6FC00E9B6F9C6B060E536EB1
:1023F0001E0E0A01B66F000153EC0AF0015201E013
:102400001A8C72EF12F0D751A508D8A4B2D0D851C7
:102410000E08D8A4AED0DA51A8080AE1DB510808AA
:1024200007E1040E0A017B6F0001FADC01C07AFAB1
:10243000DA51B7080AE1DB51800807E1030E0A010F
:102440007B6F0001EDDC01C07AFADA51CD080AE1B8
:10245000DB51100807E1050E0A017B6F0001E0DC8B
:1024600001C07AFADA51AC080DE1DB51E0080AE16B
:102470000A01B76BD70EB66F060EB86F0001F6DC17
:10248000015200E0DA51C60806E1DB51D00803E151
:10249000DDC07BFA2BDDDA519F0806E1DB51C00875
:1024A00003E1DDC07BFA25D5DA51CC0804E1DB512C
:1024B000E80801E125DDDA2D02D0DB2D00D0DA516C
:1024C000C60804E1DB51580801E1A9D5DA516D08CD
:1024D00009E1DB51C00806E1000E18B0010E010849
:1024E00001E145D7000E18BC010E000A03E1000E01
:1024F000016E41D0DA51730839E1DB51D80836E179
:102500000A01B76BD70EB66F060EB86F0001AEDCCE
:1025100001522CE037EC0AF0015202E04CEC0AF0D8
:10252000A50E976F0E0E986F996B860E9A6F200E00
:102530009B6F080E9C6F32C19DF033C19EF034C179
:102540009FF035C1A0F036C1A1F037C1A2F038C16B
:10255000A3F039C1A4F00E0E536E1E0E0A01B66F21
:10256000000153EC0AF0015201E01A8C010E016ED9
:1025700002D0000E016EFFEF13F0000E18B4010E32
:10258000010803E1010E016E02D0000E016E11EF91
:1025900014F01A8877EF14F0C68A979A8E8A989862
:1025A0008F888C82180E0A017A6F7ACA31F09E9059
:1025B0003150FD0802E2FD0E316E3150CF5CFDE37B
:1025C000CEA6FED7CECF22F022A001D002D00000AE
:1025D000000022A201D003D000000000000022A4CD
:1025E00001D005D000000000000000000000000045
:1025F000CC6A9E929EA2FED7CCCF22F022A001D020
:1026000002D00000000022A201D003D00000000090
:10261000000022A401D005D000000000000000004E
:10262000000000006B9A6B986B88A4BA6E50A4BA35
:102630006E50640E286E988486A404D0285202E05E
:102640002806F9D7988486B404D0285202E02806D8
:10265000F9D7988486A404D0285202E02806F9D736
:10266000988486B404D0285202E02806F9D7080ED0
:10267000006E002EFED76B9A6B986B88A4BA6E50D2
:10268000A4BA6E50A4AAFED76E50016E01C022F00B
:10269000206A1E0E286E285214E02050CA0811E04D
:1026A000D8902036A4AAFED76E50016E01C022F049
:1026B0002250E709FF0802E1208001D0209028067F
:1026C000EAD72050CA0803E0000E016E15D10001C0
:1026D000F5EC07F020C029F0F5EC07F020C077FA00
:1026E00077EC08F020C02BF077EC08F020C02CF03D
:1026F000246A51EF09F018AA02D0010E246E245268
:1027000005E1000E016E0A01F7D00001286A285089
:102710000B080DE377EC08F0036A28502F0FE96EE1
:10272000010E0320EA6E20C0EFFF282AF0D70C0E1E
:102730000A01775DFE0F2D6E2D50400803E2000E5A
:10274000016EDAD0286A2D50285C0FE2000177EC88
:1027500008F0036A2850D70FE96E000E0320EA6ED6
:1027600020C0EFFF282A0A01EED7286A2850010866
:102770000FE3000177EC08F0036A28503F0FE96E81
:10278000010E0320EA6E20C0EFFF282A0A01EED7CF
:10279000010EB86F2F0EB76FBA6BD70EB96F2DC081
:1027A000BBFA0001B8EC09F002C079FA01C078FA6E
:1027B0000A017951036A01013F19286E40510A014B
:1027C0007819006E7951036E00502812285206E0E5
:1027D0000101416B000E016E0A018ED00001D7513C
:1027E000A5080DE1D8510E080AE1000E18BE010E31
:1027F000000A05E1010E0101416F000104D6D75125
:10280000A5080AE1D8510E0807E1000E010194B1B4
:10281000010E01086EE10001020E0101416F00018D
:10282000ACD6015265E1286A28500B081DE3036A03
:102830002850170F016E010E032201500A017A6F12
:1028400003C07BFA036A28502F0FE96E010E0320A4
:10285000EA6EEF507C6F7BCAEAFF7ACAE9FF7CCA56
:10286000EFFF282A0001E0D7286A2D50285C1DE2DE
:10287000036A2850570F016E000E032201500A010F
:102880007A6F03C07BFA036A2850D70FE96E000EF7
:102890000320EA6EEF507C6F7BCAEAFF7ACAE9FF39
:1028A0007CCAEFFF282A0001E0D7286A28500108D7
:1028B0001DE3036A28503B0F016E010E03220150F5
:1028C0000A017A6F03C07BFA036A28503F0FE96E52
:1028D000010E0320EA6EEF507C6F7BCAEAFF7ACAD2
:1028E000E9FF7CCAEFFF282A0001E0D752D61886FC
:1028F0000101010E016E0A010001EBEF1BF08B8458
:10290000000C979C8E8C000C1AA803D0010E016E4F
:1029100002D0000E016EB0EF14F01AAA03D0010E1F
:10292000016E02D0000E016E97EF14F0F6D7015041
:10293000BAEF14F0465200E1465206E03FA202D040
:10294000DEDF02D002EC00F0462C06D01B2C02D0B9
:10295000D8DF02D07DEC0FF04650030807E1D4D752
:10296000015202E0CEDF02D07DEC0FF046500208AB
:1029700007E1DCD7015202E0C4DF02D07DEC0FF0AA
:10298000465006081BE101014151020A000105E021
:10299000030A07E0010A09E00CD0B3DF02EC00F003
:1029A0000DD0AFDF02EC00F009D07DEC0FF0A7DF17
:1029B00005D07DEC0FF002EC00F000D006EF1CF02B
:1029C0001FBE502A1FBC4F2A1FBA4E2A1FB84D2ABD
:1029D0001FB64C2A1FB44B2A1FB24A2A1FB0492ADD
:1029E000512A513C42D0246AFF0E286E296A295090
:1029F00007081BE3036A2950490FE96E000E032004
:102A0000EA6EEF50226E22507F0803E2800E225EB3
:102A100003D0800ED88022562850225C04E229C0C0
:102A200024F022C028F0292AE2D7036A24506BEC54
:102A300001F0016E01C048F0036A245077EC01F008
:102A40000A01776F77CA7BFA000176EC0FF0246AEF
:102A5000245008080AE3036A2450490FE96E000E67
:102A60000320EA6EEF6A242AF3D711EF1CF037EC4B
:102A70000AF001520AE05206525207E11A901AACCB
:102A800002D01A9C01D01A92536A1AEF1CF037EC4C
:102A90000AF0015204E0010E016E04D003D0000ED2
:102AA000016E00D0000C80EC0FF0000CFCDF000C7D
:102AB000080E0A019C6F00C09DFA958C0000958657
:102AC00083A6FED783BCD88083ACD89001360000A3
:102AD00095968C969C2FF1D7958C00008C9C9D51DF
:102AE000D8A4959C0000958683A6FED700008C96FE
:102AF000959600008C9C959C0001000C9ACA00F0F1
:102B0000D7DF0150000C0A01956B946B00010BECB0
:102B10000CF0A00E0A01CB6F00013FEC0CF001524B
:102B200005E044EC0CF0010E016E7BD00A0EE8CFFC
:102B3000EAFF8F0EE96EEFCF96FA96CACBFA3FEC1A
:102B40000CF0015205E044EC0CF0020E016E69D06D
:102B50000A0EE8CFEAFF8E0EE96EEFCF96FA96CA1C
:102B6000CBFA3FEC0CF0015205E044EC0CF0040E03
:102B7000016E57D00BEC0CF0A10E0A01CB6F0001D7
:102B80003FEC0CF0015205E044EC0CF0080E016E35
:102B900048D00A01956B946B010E925D006E000E99
:102BA0009359036E0050016E9551035C1DE303E1E0
:102BB0000150945D19E290519425016E9151952137
:102BC000036E0150966F03C097FA010E9A6F0001D1
:102BD00095DF97CAEAFF96CAE9FF01C0EFFF0A0135
:102BE000942BD8B4952BD8D7010E925D966F000E1A
:102BF0009359976F90519625016E91519721036ECD
:102C00000150986F03C099FA9A6B000177DF99CA57
:102C1000EAFF98CAE9FF01C0EFFF44EC0CF0000E98
:102C2000016E000C0A019051E96E91CAEAFFEF5063
:102C3000946F9251E96E93CAEAFFEF50956F95CA6F
:102C400096FA94CA95FA96CA94FA8F51951B9539BB
:102C5000006E0F0E00160050951B9539006EF00E99
:102C600000160050941B9531006E003200321F0E8A
:102C700000160050941B9539006EF00E001600509F
:102C8000D89000360050951B9051E96E91CAEAFF2A
:102C900094CAEFFF9251E96E93CAEAFF95CAEFFF1B
:102CA0000001000C8ECA44F08D80200E286E285240
:102CB00006E098908F8098908F902806F8D78D9096
:102CC0000A018E5308E098908F8098908F908E071D
:102CD0000001F6D70A010001000C020E1B6E979A44
:102CE0008E9A98988F988C9498968F860A018F6BFD
:102CF0005A0E8E6F8E518F1125E0FA0E906FD8907C
:102D0000903390519007000AFCE1FA0E906FD89032
:102D1000903390519007000AFCE1FA0E906FD89022
:102D2000903390519007000AFCE1FA0E906FD89012
:102D3000903390519007000AFCE18E51D8B48F0770
:102D40008E07D8D744C08EFA0001ACDFD8DD0A0167
:102D50008F6BC80E8E6F8E518F1125E0FA0E906F1B
:102D6000D890903390519007000AFCE1FA0E906FD2
:102D7000D890903390519007000AFCE1FA0E906FC2
:102D8000D890903390519007000AFCE1FA0E906FB2
:102D9000D890903390519007000AFCE18E51D8B43E
:102DA0008F078E07D8D7000102EC00F00A018F6B65
:102DB000C80E8E6F8E518F1125E0FA0E906FD8904D
:102DC000903390519007000AFCE1FA0E906FD89072
:102DD000903390519007000AFCE1FA0E906FD89062
:102DE000903390519007000AFCE1FA0E906FD89052
:102DF000903390519007000AFCE18E51D8B48F07B0
:102E00008E07D8D71A8E9E90FD0ECF6EE80ECE6E2E
:102E1000CC6A9D800001000C60DF000C47DE6FDD96
:102E200070DD0A01786B796B01019E6B400E9D6F1E
:102E3000A76BA66BC00EA56FA46B000109EC0CF08C
:102E40000A018F6B8E6B0A0E916F7E0E906F936BE3
:102E5000100E926F000157DE0A0EE8CFEAFF7D0EDA
:102E6000E96E80CAEFFF0A0EE8CFEAFF7C0EE96E3A
:102E700081CAEFFF0A017B6B7A6B7B517D5D59E361
:102E800003E17C517A5D55E27B51070818E303E1C9
:102E90007A51930814E39EC18FFA9DC18EFA0A0EEF
:102EA000916F7E0E906F936B100E926F00012BDE70
:102EB000100E01019D27000E9E231AD00A01A6C103
:102EC000F8FFA5C1F7FFA4C1F6FF0A0EEA6E7E0E59
:102ED000E96E100E006E0900F5CFEEFF002EFBD755
:102EE000F86A100E0101A427000EA523A623A7232C
:102EF0000A01776B77510F0818E3036A77517E0F49
:102F0000E96E0A0E0320EA6EEFCF8EFA8ECA8FFAB0
:102F10000A0E916F780E906F0A0E936F790E926F72
:102F2000000180DE0A01772BE5D77A2BD8B47B2B02
:102F3000A4D7A2C18FFA0A0E916F780E906F0A0E75
:102F4000936F790E926F00016DDEA3C18FFA0A0EA6
:102F50000A01916F780E906F0A0E936F790E926F3F
:102F6000000160DE59DF0A01785306E1795304E17C
:102F7000010E016E04D003D0000E016E00D00001DE
:102F8000F0EF17F093DDF29CF29EF2BEFDD780EFDA
:102F90005EF030EF18F0000E010194B5010E000A4A
:102FA000D8A4AED096519A5D5DE303E19951955D49
:102FB00059E200016CDD0152D8B402D0010152D0B7
:102FC0000101A1510E0845E3000137EC0AF001525E
:102FD00002E04CEC0AF00101A15309E100011ED707
:102FE00001B003D00101949302D001019483A50E96
:102FF0000001976F0E0E986F996BC60E9A6F580E60
:103000009B6F030E9C6F010194A311D0010EE8CFBA
:10301000EAFF9C0EE96EEF5000019D6F010EE8CFB4
:10302000EAFF9B0EE96EEF509E6F05D00101CC0EBA
:1030300000019D6F9E6F080E536E1E0E0A01B66F43
:10304000000153EC0AF0015201E01A8C0101A12B9E
:1030500008D094A302D0000195D700018EEC0FF0A8
:1030600001014AD0995302E19A5346E0A051640805
:1030700005E200018EEC0FF040D001019F510508E0
:1030800035E2000104DD0152D8B402D001012ED096
:1030900037EC0AF0015202E04CEC0AF0A50E976FF3
:1030A0000E0E986F996BC60E9A6F580E9B6F020E9C
:1030B0009C6F010EE8CFEAFF9C0EE96EEF509D6F0A
:1030C000010EE8CFEAFF9B0EE96EEF509E6F080EEF
:1030D000536E1E0E0A01B66F000153EC0AF0015246
:1030E00001E01A8C01019F6BA02B06D00001CFDC00
:1030F000015203E101019F2B00010101949501D0D0
:10310000949500011CEF1CF0000E18B6010E01088A
:1031100003E1010E016E02D0000E016E91EF18F076
:10312000F3D70150C9EF19F00A017B6B020E0101C0
:10313000185D0A017B5D01E022E2036A7B51570FB3
:10314000E96E000E0320EA6E7951EF5C16E1010E84
:103150007B25036A570FE96E000E0320EA6E7A5151
:10316000EF5C0BE1020E7B25036A570FE96E000E40
:103170000320EA6EEF50016E04D07B2BD7D7FF0EF1
:10318000016E0001C9EF18F077CA79FA78CA7AFAA5
:10319000CBD70150FF0804E0010E016E04D003D02C
:1031A000000E016E00D0D2EF19F00A017E6B020E04
:1031B0000101185D0A017E5D01E02BE2036A7E5188
:1031C000570FE96E000E0320EA6E7C51EF5C1FE1A1
:1031D000010E7E25036A570FE96E000E0320EA6E8A
:1031E0007D51EF5C14E1020E7E25036A570FE96EF4
:1031F000000E0320EA6EEF520AE0030E7E25036AFA
:10320000570F016E000E03220350026E02D07E2B78
:10321000CED70001000C3BDC015202E04CEC0AF07E
:10322000A50E0A017F6F0E0E806F00015BEC0EF0A1
:103230006C0E0A017F6F800E806F00015BEC0EF058
:103240000A01776B7751070812E3030E7725036AAB
:103250002F0FE96E010E0320EA6EEFCF79FA79CADB
:103260007FFA000195EC0EF00A01772BEBD7660E82
:103270007F6F400E806F00015BEC0EF0010E0A01C3
:103280007F6F000195EC0EF0660E0A017C6F400E18
:103290007D6F00018ADF02C079FA01C078FA010E61
:1032A0000A010124016E000E0220036E0150E96E36
:1032B00003C0EAFFEFCF7AFA7ACA7FFA000195ECF1
:1032C0000EF0140E0A017F6F0001C1EC0EF0FAEF50
:1032D00019F00101DB91DB97D96BAD6BAE6BDB991C
:1032E0000001000C0A01796B0101DBA14ED0020E36
:1032F000D95DF80FFD0F0A01786F776B77510708DA
:1033000018E377517825036AB10FE96E010E0320A7
:10331000EA6EEFCF7BFA030E7725036A2F0FE96E73
:10332000010E0320EA6EEF507B5DD8B4792B772B2A
:10333000E5D77951080828E10C0E7825036AB10F0A
:10334000E96E010E0320EA6EEFCF7BFA660E7C6F0A
:10335000400E7D6F000129DF02C07DFA01C07CFABA
:10336000010E0A010124016E000E0220036E0150BD
:10337000E96E03C0EAFFEF507B5D06E10101DB83EC
:10338000DB850001A6DF0A01010100010BEF1AF045
:10339000C7D6015240E0660E0A01776F400E786F83
:1033A0000001F2D6015237E06C0E0A017C6F800EEC
:1033B0007D6F0001FADE02C078FA01C077FA02C020
:1033C000B7FA01C0B6FA0A01B86B000136EC0FF08B
:1033D000015221E0660E0A017C6F400E7D6F0001F4
:1033E000E4DE02C003F00150E96E02C0EAFFEF52D2
:1033F00002E111D710D0660E0A017C6F400E7D6F7E
:103400000001D3DE02C003F00150E96E02C0EAFF02
:10341000EF2C01D067D7A8EF1AF00101F76B0A0172
:10342000776B7751020814E37751090DF350796BEC
:10343000786F080E7825016E000E7921036E015019
:10344000DC0FE96E010E0320EA6EEF6A772BE9D7F5
:103450000101B06BAF6B0001000C0101DBA10DD0CD
:10346000AD530BE0AD07AD5308E1AE07AE5304E03A
:10347000DB87320EAD6F01D0DB89AF51B0110AE0AE
:10348000AF51D8B4B007AF07AF51B01103E100019D
:10349000C4DF01010001A9EF1AF037EC0AF0015274
:1034A00003E0000E016E17D0000E18B8010E0108DF
:1034B00003E1000E016E0FD0400E016E010EEA6EA8
:1034C000420EE96EEE6A012EFDD70101826B936B0D
:1034D000010E016E00016EEF1AF0DFD7010EEA6EE9
:1034E000420EE96E010EE26EB10EE16E0101D9519C
:1034F000016E04E0E6CFEEFF012EFCD7D9C182F1C8
:103500000A0E0A017F6F0001C1EC0EF094EF1AF071
:103510000101DBA70AD0000147EC15F0015204E1DC
:103520000101DB970001D9D701010001AAEF1AF0D0
:103530000101DBA904D00001CCDE0101DB93000115
:10354000ABEF1AF0010194AB07D0DB95000120D757
:1035500084D7DED7EDD701010001B0EF1AF0F2D722
:1035600029EF1CF000D0010E196E1A9A1896030E5E
:103570000101416F000189EF01F0C3EF01F001C0CB
:103580001FF09E90C68A040E6F6E6C946C886C8ED1
:103590006C9C6B8E6B9A6B9C6B986C9A6B8E979AEB
:1035A0008E8A98988F888C821B50630801E11ED008
:1035B0001B50020801E104D01B2C01D08BD04ED14E
:1035C000060E196E9D90979A8E8A98988F888C8295
:1035D00041EF04F0015205E0010E1B6E1E6AB5D0EA
:1035E00004D0CF6A960ECE6EF9D0F8D0630E196E65
:1035F0009D90979A8E8A98988F888C820A01786B12
:10360000010E796F0001EFEC01F001C022F02252AF
:1036100060E0979A8E9A98988F88CF500E0801E2B2
:10362000DDD00F0E0A017A6F7ACA31F09E903150C8
:10363000FD0802E2FD0E316E3150CF5CFDE3CEA6F7
:10364000FED7CECF22F022A001D002D00000000091
:1036500022A201D003D000000000000022A401D06B
:1036600005D0000000000000000000000000CC6A4F
:103670009E929EA2FED7CCCF22F022A001D002D0F3
:103680000000000022A201D003D0000000000000D2
:1036900022A401D005D000000000000000000000BE
:1036A0000000AA0E326EC950206E3250C96EC7A0FB
:1036B000FED726C032F0C950206E3250C96EC7A066
:1036C000FED7326AC950206E3250C96EC7A0FED7ED
:1036D000000184D0020E196E1D502E5C0AE21E50AD
:1036E000040807E3979A8E9A98988F88BFEC03F0A6
:1036F00014D0979A8E8A98988F888C820A0E0A0125
:10370000786F010E796F0001EFEC01F001C022F03B
:10371000225202E01E6A01D01E2A00D0030E196E4A
:1037200018922EAA0CD0010E0A01776F00018DECC1
:1037300004F001C01FF01E5201E1188205D00A01F9
:10374000776B00018DEC04F000D0040E196E0A01B5
:10375000C16B2FC0C0FA010EC36FC26B000186ECB3
:1037600005F002C042F001C041F02E504126000E8B
:103770004222CF500E0801E231D01AA010D042C030
:1037800078FA41C077FA97EC05F001C020F0202CC0
:1037900001D00FD02050020801E115D009D00A0154
:1037A000786B776B000197EC05F0015201E00BD0CC
:1037B00015D0050E196ECF50170801E20FD05FEF3C
:1037C00006F0E8EF07F0080E196ECF50170801E277
:1037D00005D0CCEF12F0015200E100D0140E196EAA
:1037E000979A8E8A98988F888C82326AC950206EF8
:1037F0003250C96E6B9E8B9AC69A979A8E9A9898F9
:103800008F983F2AD8B4402A9AEF14F01B2C05D089
:103810001E50070802E2020E1B6E18A202D0E0EF53
:1038200014F09E901AAE02D09D8002D080EC0FF072
:1038300037EF15F0CBEF17F0050E0A01906FD89017
:10384000903390519007000AFCE118B003D00001BA
:1038500086D60A01000E016E09D000010A0E196E0B
:103860007FEC14F002EC00F0B9D70A019E90000141
:103870002AEF00F0010E0101F86FFA6FFB6BFE6B8F
:10388000F96FFD6FFC6F000122EF2BF0D8900A0159
:103890000535036A330FE96E000E0320EA6E07CA8E
:1038A000ECFFED5206CAEFFF0001000CC26A0D0EDC
:1038B000C16E060EC06E32EF1DF00A010551000AFE
:1038C000000105E0010A1AE0030A2FE03ED0EF0EE6
:1038D000926E806AFF0E936E816ADB0E946E826A2E
:1038E0007A0E956E040E836E0C0E966E846A1B0E15
:1038F000976E856AE40E986E866A27D0D30E926E14
:10390000806AFF0E936E816ADB0E946E826A020EED
:10391000956E040E836E0C0E966E846A1A0E976E68
:10392000856AE40E986E866A10D0FF0E926E806EE5
:10393000936E816E946E826E956E836E966E846EBB
:10394000976E856E986E866E00D0000E016E36EF13
:103950001DF00A010751F90F21E2070F0001D0EF16
:103960001CF00F0EC16E0A0119D00E0EC16E0A01B5
:1039700015D00E0EC16E0A0111D00E0EC16E0A01D5
:103980000DD00E0EC16E0A0109D00E0EC16E0A01D5
:1039900005D00E0EC16E0A0101D00A010001000C13
:1039A000F2CF0EF0F29EE824C50FF66E390EF76ED8
:1039B000D8B0F72A0A00F550FA6E0800F5500EBE8E
:1039C000F28EF96E62396A3972397A3982398A39F6
:1039D0009239C150F00B0A01066F0551FB0F28E226
:1039E000050F00011AEF1DF0020E0A01076F00011A
:1039F000B0DF0A011DD0030E0A01076F0001A9DF25
:103A00000A0116D0040E0A01076F0001A2DF0A01A5
:103A10000FD0050E0A01076F00019BDF0A0108D0D5
:103A2000060E0A01076F000194DF0A0101D00A01A6
:103A30000001000CF2CF0EF0F29EE824590FF66E52
:103A40003A0EF76ED8B0F72A0A00F550FA6E080061
:103A5000F5500EBEF28EF96EE839F639043A123A94
:103A6000203A24D70A01056B000127D70A01056B0C
:103A70000001AFDF04EC0CF0176AF2BE178EF29E65
:103A800009EC0CF017BEF28E189051EF2BF0030EDC
:103A90000A01056F00019DDF93948A8493869388C1
:103AA00093948A84938A939C8A8C93948A84978033
:103AB000938E93948A849780938E95988C8892861F
:103AC00095988C88928493928A8293948A84978022
:103AD000938E53EF2BF00A01096B0951070825E378
:103AE000D89009350B6B0A6F830E0A25E96E010E1B
:103AF0000B21EA6E0751EF5C16E1D89009350E6B89
:103B00000D6F010E0D25016E000E0E21036E01508A
:103B1000830FE96E010E0320EA6E0851EF5C03E1AA
:103B2000010E016E49D0092BD8D7096B095107083E
:103B300041E3D89009350B6B0A6F830E0A25E96EB5
:103B4000010E0B21EA6EEF5233E1D89009350E6B6E
:103B50000D6F010E0D25016E000E0E21036E01503A
:103B6000830FE96E010E0320EA6EEF5221E1D89037
:103B700009350B6B0A6F830E0A25E96E010E0B21C6
:103B8000EA6E07CAEFFFD89009350B6B0A6F010E7A
:103B90000A25016E000E0B21036E0150830FE96EA2
:103BA000010E0320EA6E08CAEFFF010E016E04D079
:103BB000092BBCD7000E016E0001E6EF1DF0A50E2B
:103BC0000A01076F0E0E086F000185D701C006FAC3
:103BD0000A010651016E000114EF1EF00A01056B87
:103BE000055107081EE3D8900535076B066F830E55
:103BF0000625E96E010E0721EA6EEF6AD8900535B9
:103C0000076B066F010E0625016E000E0721036E7D
:103C10000150830FE96E010E0320EA6EEF6A052B57
:103C2000DFD7189A0001CBD7000E016E48EF1FF0C6
:103C30008EEC0FF053EF1FF005CA46F00A01055352
:103C400006E100017DEC0FF002EC00F00A0100013A
:103C500058EF1FF02F6A0A01056B0551070810E3A2
:103C6000176AF2BE178EF29E05CA7FFA0001AFEC0A
:103C700011F017BEF28E01502F1A0A01052BEDD755
:103C80002F5202E18D0E2F6E2FC047F0000180EF02
:103C90001EF0979A9898949A988495949592979AEA
:103CA0008E9A98988F988C8498968F96850ECD6E64
:103CB000CD9E080E016E0409CA6E130ECB6ECD9612
:103CC000040E6F6E6C946C886C8E6C9C6B8E6B9A11
:103CD0006B9C6B986C9A6B9EC69A230EC66E000EF8
:103CE000C76E326AC950206E3250C96EC7A0FED767
:103CF000326AC950206E3250C96E8B9AC69AAAD7C2
:103D0000800E1A6E010E1C6E500E1D6E020E456E58
:103D1000200E446E406A3F6A436A246A24500808B1
:103D20000AE3036A2450490FE96E000E0320EA6E8D
:103D3000EF6A242AF3D73AEF1FF00A01076B056BED
:103D4000055107081DE3176AF2BE178EF29E05CAD9
:103D50007FFA0001AFEC11F017BEF28E01C006FA37
:103D6000030E0A010525036A230FE96E010E0320E5
:103D7000EA6E06CAEFFF063D01D0072B052BE0D700
:103D80000751070818E3176AF2BE178EF29E790EE4
:103D9000C36F880EC26F010EC56F260EC46FC76B4E
:103DA000080EC66F000171EC0CF017BEF28E010E0A
:103DB000016E53D00A01176AF2BE178EF29E790E79
:103DC0008F6F880E8E6F010E916F260E906F936B22
:103DD000080E926F000183EC15F017BEF28E0A01F7
:103DE000076B056B055107080FE3030E0525036AF2
:103DF000230FE96E010E0320EA6EEF50066F063DB9
:103E000001D0072B052BEED70751070823E3056BDD
:103E1000055107081AE3030E0525036A230FE96E0F
:103E2000010E0320EA6EEFCF09FA176AF2BE178E71
:103E3000F29E05CA7EFA09CA7FFA00019DEC11F0D4
:103E400017BEF28E0A01052BE3D7010E016E0001A9
:103E500004D00A01000E016E00013BEF1FF0546A0E
:103E6000050E0101236F536A18941896030E416FD3
:103E700000010FD762D7B7EF1FF0176AF2BE178E97
:103E8000F29E56EC15F017BEF28E7FEC14F0A6D61B
:103E900018980101936B189A188C189E9491826B54
:103EA000936B0001C5D6010E0A01056F0001C4D64F
:103EB0007FEC14F00A018F6BC80E8E6F8E518F113C
:103EC00025E0FA0E906FD890903390519007000A39
:103ED000FCE1FA0E906FD890903390519007000A51
:103EE000FCE1FA0E906FD890903390519007000A41
:103EF000FCE1FA0E906FD890903390519007000A31
:103F0000FCE18E51D8B48F078E07D8D7000102ECA0
:103F100000F00A018F6BC80E8E6F8E518F1125E055
:103F2000FA0E906FD890903390519007000AFCE100
:103F3000FA0E906FD890903390519007000AFCE1F0
:103F4000FA0E906FD890903390519007000AFCE1E0
:103F5000FA0E906FD890903390519007000AFCE1D0
:103F60008E51D8B48F078E07D8D7000178D7176A3B
:103F7000F2BE178EF29E0CEC17F017BEF28E57EFC2
:103F80002BF0189E0A0105B1188E010194910A01C7
:103F900006A103D0010194810A010001E2EF1FF0A4
:103FA00069EC19F0176AF2BE178EF29E0DEC1AF04A
:103FB00017BEF28EE3EF1FF00A01056B010E066FCC
:103FC0000001DFD7EDD70101DB93948B000159EF9E
:103FD0002BF0188A5BEF2BF05DEF2BF05FEF2BF0EF
:103FE0000BEC0CF0176AF2BE178EF29EA00E0A01BF
:103FF000CB6F00013FEC0CF017BEF28E015205E0D2
:1040000044EC0CF0010E016E60D00A0EE8CFEAFF1E
:10401000080EE96EEFCF0BFA176AF2BE178EF29E0A
:104020000BCACBFA3FEC0CF017BEF28E015205E042
:1040300044EC0CF0020E016E48D00A0EE8CFEAFF05
:10404000070EE96EEFCF0BFA176AF2BE178EF29EDB
:104050000BCACBFA3FEC0CF017BEF28E015205E012
:1040600044EC0CF0020E016E30D00BEC0CF0176A31
:10407000F2BE178EF29EA10E0A01CB6F00013FEC3B
:104080000CF017BEF28E015205E044EC0CF0030E6A
:10409000016E1BD00ACA03F00A0109510B6F0ACA4C
:1040A0000CFA176AF2BE178EF29E9A6B00017EEC34
:1040B00015F017BEF28E0CCAEAFF0BCAE9FF01C069
:1040C000EFFF44EC0CF0000E016ED3EF23F00A0179
:1040D000646B43CA03F04251E96E43CAEAFFECCF76
:1040E00066FAED52EFCF65FA6631686F6531676F3A
:1040F00068336733683367336833673368336733EC
:10410000070E68170901F6510A01675D05E109010B
:10411000F7510A01685D79E04251E96E43CAEAFF4E
:10412000ECCF66FAED52EFCF65FA66310901F76F11
:104130000A0165310901F66FF733F633F733F633C9
:10414000F733F633F733F633070EF7170A01425108
:10415000E96E43CAEAFFECCF66FAED52EFCF65FA9B
:1041600065511F0B0901F86F176AF2BE178EF29E98
:10417000000109EC0CF017BEF28E43CA03F00A01ED
:104180004251E96E43CAEAFFECCF66FAED52EFCF37
:1041900065FA176AF2BE178EF29E66CA8FFA65CA72
:1041A0008EFA0A0E916F440E906F936B200E926FF1
:1041B000000183EC15F017BEF28E036A0901F85175
:1041C000440FE96E0A0E0320EA6EEF500A01646F95
:1041D0004251656F4251E96E43CAEAFFECCF68FA7B
:1041E000ED52EFCF67FA010E6725016E000E6821D0
:1041F000036E0150696F43CAEAFF65CAE9FF03C055
:10420000ECFFED5269CAEFFF33D04251E96E43CA69
:10421000EAFFECCF66FAED52EFCF65FA65511F0B5E
:104220000901F86F036AF851440FE96E0A0E032082
:10423000EA6EEF500A01646F4251656F4251E96EB8
:1042400043CAEAFFECCF68FAED52EFCF67FA010EEE
:104250006725016E000E6821036E0150696F43CA25
:10426000EAFF65CAE9FF03C0ECFFED5269CAEFFF40
:104270006451016E0001000C0A013A6B0701E56B05
:10428000040EE66F0A01375304E136513A5DD8B0A7
:1042900004D10A0E436F340E426F000118DF01C0D3
:1042A0003FFA0A013A2B0A0E436F340E426F0001A7
:1042B0000EDF01C03BFA0A013A2B3F531DE1386B78
:1042C0003B51385D19E2036A3851BC0F016E080E8C
:1042D00003220150406F03C041FA0A0E436F340EAF
:1042E000426F0001F4DE41CAEAFF40CAE9FF01C0A3
:1042F000EFFF0A01382BE4D73F2D8AD0386B396B9A
:104300003B51385DD8B084D00A0E436F340E426FF3
:104310000001DDDE01C03CFA0A01382B3C510E08D9
:1043200003E03C510F0815E10A0E436F340E426F53
:104330000001CDDE01C03DFA0A01382B0A0E436FA1
:10434000340E426F0001C3DE01C03EFA0A01382B71
:104350003CD03C51140815E10A0E436F340E426FF5
:104360000001B5DE01C03DFA0A01382B0A0E436F89
:10437000340E426F0001ABDE01C03EFA0A01382B59
:1043800024D03C510D080BE10A0E436F340E426FEE
:1043900000019DDE01C03DFA0A01382B16D03C51C8
:1043A000100809E03C51110806E03C51120803E0F6
:1043B0003C5113080AE10A0E436F340E426F0001AC
:1043C00086DE01C03DFA0A01382B3951392B416F85
:1043D000176AF2BE178EF29EC16B41CAC0FAC36B58
:1043E000030EC26F000186EC05F017BEF28E01507D
:1043F000090FE96E020E0220EA6EEE523ECAECFF91
:10440000ED523DCAEFFFED523CCAEFFF0A0178D7EB
:104410003F5102081DE1386B3B51385D19E2036AD8
:104420003851F40F016E070E03220150406F03C094
:1044300041FA0A0E436F340E426F000148DE41CA52
:10444000EAFF40CAE9FF01C0EFFF0A01382BE4D7B9
:104450003F5103081DE1386B3B51385D19E2036A97
:104460003851580F016E080E03220150406F03C0EF
:1044700041FA0A0E436F340E426F000128DE41CA32
:10448000EAFF40CAE9FF01C0EFFF0A01382BE4D779
:104490003B513A270701F6D60A01000E016E0001D2
:1044A000B8EF23F00A01316BD89002010735036A97
:1044B000FF0FE96E010E0320EA6EECCF03F0ED5220
:1044C000EF500A01276F03C028FA200E016E0A0E72
:1044D000EA6E070EE96EEE6A012EFDD7176AF2BE8C
:1044E000178EF29E000109EC0CF017BEF28E176ACF
:1044F000F2BE178EF29E50EC0CF017BEF28E0152F7
:1045000001E1F5D7176AF2BE178EF29E28CA8FFA1C
:1045100027CA8EFA0A0E0A01916F070E906F936BED
:10452000200E926F000183EC15F017BEF28E01C0D1
:1045300031FA200E0A012727000E282307CA2BFA7A
:1045400008CA2CFA09CA2DFA0ACA2EFA2F6B306B48
:104550002C5301E02B07326B2B51325D35E2176A89
:10456000F2BE178EF29E28CA8FFA27CA8EFA0A0E5A
:10457000916F070E906F936B200E926F000183EC8A
:1045800015F017BEF28E01500A013113176AF2BE00
:10459000178EF29E0A0EC36F070EC26F200EC46FF5
:1045A0000A0EC66F2F0EC56F0A0EC86F300EC76F8A
:1045B0000001A1EC0BF017BEF28E200E0A01272796
:1045C000000E2823322BC8D72C535FE0176AF2BEA7
:1045D000178EF29E28CA8FFA27CA8EFA0A0E916F9A
:1045E000070E906F936B2CCA92FA000183EC15F0C2
:1045F00017BEF28E01500A013113176AF2BE178EF0
:10460000F29E0A0EC36F070EC26F2CCAC4FA0A0EBE
:10461000C66F2F0EC56F0A0EC86F300EC76F000130
:10462000A1EC0BF017BEF28E176AF2BE178EF29E47
:104630000A0E0A01C36F2D0EC26F010EC46F0A0E5F
:10464000C66F2F0EC56F0A0EC86F300EC76F000100
:10465000A1EC0BF017BEF28E176AF2BE178EF29E17
:104660000A0E0A01C36F2E0EC26F010EC46F0A0E2E
:10467000C66F2F0EC56F0A0EC86F300EC76F0001D0
:10468000A1EC0BF017BEF28E0A01176AF2BE178E6C
:10469000F29E600E7F6F780E806F00015BEC0EF073
:1046A00017BEF28E176AF2BE178EF29E2FCA7FFADD
:1046B00095EC0EF017BEF28E176AF2BE178EF29EC0
:1046C00030CA7FFA95EC0EF017BEF28E176AF2BE72
:1046D000178EF29E07C27FFA95EC0EF017BEF28E8F
:1046E000176AF2BE178EF29E31CA7FFA95EC0EF071
:1046F00017BEF28E176AF2BE178EF29E140E0A01D2
:104700007F6F0001C1EC0EF017BEF28E0A0131532B
:1047100003E03151016E2FD02F5302E1305303E0FB
:10472000100E016E28D02B51200DF3502C25296F2F
:104730002A6BD89002010735036AFF0FE96E010E5C
:104740000320EA6EECCF35FAED52EFCF34FA200EAB
:104750000A013425276F000E3521286F28CA35FA43
:1047600027CA34FA2ACA37FA29CA36FA000184D588
:10477000000E016E0A010001000C0A01056B066BB8
:10478000176AF2BE178EF29E000109EC0CF017BEFC
:10479000F28E300E0A01086F076B0A0E0A6F050EC3
:1047A000096F00011DD401520EE1020108510A01F6
:1047B000055D07E205CA07F2000174DE01C006FAD2
:1047C0000A0104D00001010E0A01066F0651016EB4
:1047D000000170EF2BF00BCA03F00A010A510C6FB5
:1047E0000901E807036AE851200FE96E090E03206A
:1047F000EA6EEF500A010E6F0BCAEAFF0CCAE9FF1E
:104800000ECAEFFF0001000C0901E851E82B036A12
:10481000200FE96E090E0320EA6E0CCAEFFF0001BB
:10482000000C0901EA51EA2B036A840FE96E090EB4
:104830000320EA6E05CAEFFF000175EF2DF00901B4
:10484000E951E92B036ABC0FE96E080E0320EA6EFA
:1048500006CAEFFFE951E92B036ABC0FE96E080EA7
:104860000320EA6E07CAEFFFE951E92B036ABC0F88
:10487000016E080E032201500A01096F03C00AFAF3
:10488000010E065D036AE50FE96E070E0320EA6E6E
:10489000EF500C6F0ACAEAFF09CAE9FF0CCAEFFF22
:1048A0000901E951E92B036ABC0F016E080E0322CE
:1048B00001500A01096F03C00AFA036A0901EB51AA
:1048C000E50FE96E070E0320EA6EEF500A010B6F49
:1048D0000ACAEAFF09CAE9FF0BCAEFFF06CAEBF9E9
:1048E000036A0901EB51E50FE96E070E0320EA6E3A
:1048F000E9C9EFFF0A0107510901E927090126EF7C
:104900002EF0036A0901EB51E50FE96E070E032053
:10491000EA6EEF500A01056F030E055D036ABC0FD6
:10492000E96E080E0320EA6EEF50096F020E055D76
:10493000036ABC0FE96E080E0320EA6EEF500A6F9F
:10494000010E055D036ABC0FE96E080E0320EA6ED6
:10495000EF500B6F0B510A5D04E10901EB072CD0FE
:104960000A010BCA06FA040E0B5D036ABC0FE96E5E
:10497000080E0320EA6EEF50076F07CA08FA090114
:10498000EB510A01085D15E3036A0851E50FE96E72
:10499000070E0320EA6E06CAEFFF020E065D036AE9
:1049A000BC0FE96E080E0320EA6EEF50066F080791
:1049B000E6D707CAEBF90901040E0A010925090126
:1049C000E95F090126EF2EF006CA03F00A0105513E
:1049D000076F0901EA07036AEA51840FE96E090EBD
:1049E0000320EA6EEF500A01096F06CAEAFF07CA00
:1049F000E9FF09CAEFFF090126EF2EF0B9EF2DF00C
:104A00000A01066B0551065D12E20A0E0B6F070ED6
:104A10000A6F0001E0DE036A0A010651970FE96E92
:104A2000000E0320EA6E07CAEFFF062BEBD705CA7C
:104A300053F0176AF2BE178EF29E140EB66F000185
:104A400053EC0AF017BEF28ECBEF2DF00A018F6BFC
:104A500005CA8EFA8E518F1125E0FA0E906FD8900C
:104A6000903390519007000AFCE1FA0E906FD890B5
:104A7000903390519007000AFCE1FA0E906FD890A5
:104A8000903390519007000AFCE1FA0E906FD89095
:104A9000903390519007000AFCE18E51D8B48F07F3
:104AA0008E07D8D7090126EF2EF08A84000CFDDF8F
:104AB000000E016E000C9780040E006E002EFED7D3
:104AC000938E060E006E002EFED78E909790040EE9
:104AD000006E002EFED78A9E939E000C080E016E7B
:104AE0000000040E006E002EFED78A9E939E060ED6
:104AF000006E002EFED70A010F378E90D8B0978037
:104B0000D8A09790938E81AEFED7012E01D002D00F
:104B10000001E6D7040E006E002EFED78A9E939EFB
:104B200000009780060E006E002EFED7060E006E67
:104B3000002EFED7938E81AEFED7016A060E006E60
:104B4000002EFED785B001808A9E939E8E9097900E
:104B50000001AEEF25F00ECA0FFAC0D70150000CCD
:104B600097900000938E81AEFED7040E006E002E4B
:104B7000FED70000000000009780040E006E002E9B
:104B8000FED7000C080E0A01106F00C011FA9780C2
:104B9000060E006E002EFED7938E81AEFED785B036
:104BA000D88085A0D8900136040E006E002EFED766
:104BB000939E8A9E102FEBD79780060E006E002ED4
:104BC000FED78E901151D8A497900000938E81AE9D
:104BD000FED7040E006E002EFED78A9E939E060E10
:104BE000006E002EFED78E9097900001FBEF25F00F
:104BF0000ECA00F0C7D70150000C5DDF900E0A010D
:104C00000E6F0001A8DF015204E0AADF020E016E60
:104C100028D00A010E6B00019EDF015204E0A0DFE4
:104C2000030E016E1ED047DF910E0A010E6F0001C8
:104C300092DF015204E094DF040E016E12D00A01EB
:104C40000E6B0001D5DF01C00DFA8ADF0A010B519E
:104C5000E96E0CCAEAFF030E0D5DEF6E000E016EE9
:104C60000001000CC2503C0B0A010C6F0B51016E8D
:104C700004E0D8900C33012EFCD70B510C5D02E000
:104C8000000E01D0010E016E0001000C000EC216D4
:104C90000A010B35006E0036FC0E00160050C212E1
:104CA000320E906FD890903390519007000AFCE13B
:104CB0000001000CF80EC016060EC012000CC280D7
:104CC000000C030E0A010B6F0001CCDF015205E15D
:104CD000030E0A010B6F0001D9DF0A010B6B000103
:104CE000E9DFEDDF000E016E87EF29F0C09EC28282
:104CF000C2B2FED7C4CF19FA0A011951016E0001E0
:104D0000000C0CCA03F00A010B510D6F0CCA0EFA0D
:104D10000001ECDF0ECAEAFF0DCAE9FF01C0EFFF98
:104D2000000E016E8EEF29F0020E0A010B6F0001DA
:104D300099DF015205E1020E0A010B6F0001A6DFA7
:104D40000A010B6B0001B6DFBADF000E016E000C2A
:104D500016CA03F00A011551176F16CA18FA000196
:104D6000C5DF18CAEAFF17CAE9FF01C0EFFF000E4E
:104D7000016E000C0A010E6B0D6B116B11517F0857
:104D80000DE30A0E166F140E156F0001E1DF0A0124
:104D900014510D27000E0E23112BF0D70E31036E88
:104DA0000D31026E0332023203320232033202321A
:104DB000033202320332023203320232010E031690
:104DC0000250126F0E6B0D6B106B0F6B116B11514C
:104DD0007F0816E30A0E166F140E156F0001B8DF78
:104DE0000A011451125D04E31451125D146F02D0D4
:104DF0001251145F14510D27000E0E23112BE7D70B
:104E00000E31036E0D31026E033202320332023272
:104E100003320232033202320332023203320232EE
:104E2000010E03160250136F0B51E96E0CCAEAFF14
:104E300013CAEFFF000E016E0001000C000E016EA0
:104E4000000C0A01176B166B196B186B81B6FED735
:104E500081A6FED781A604D0162BD8B4172BFAD77B
:104E600081B604D0182BD8B4192BFAD71251E96E99
:104E700013CAEAFF17CAECFFED5216CAEFFF14512E
:104E8000E96E15CAEAFF19CAECFFED5218CAEFFF26
:104E9000000E016E0001AAEF27F015CA19FA14CA14
:104EA00018FA17CA1BFA16CA1AFA0A011A51182553
:104EB000226F1B511921236FD89023311D6F22318E
:104EC0001C6F176AF2BE178EF29E300EBB6FD40EA7
:104ED000BA6F1DCABDFA1CCABCFA0001C3EC0FF0C0
:104EE00017BEF28E02C01FFA01C01EFA0A011C5141
:104EF000185D226F1D511959236F176AF2BE178E64
:104F0000F29E23CAC1FA22CAC0FA1FCAC3FA1ECA35
:104F1000C2FA000186EC05F017BEF28E02C021FA3B
:104F200001C020FA1251E96E13CAEAFF21CAECFF50
:104F3000ED5220CAEFFF000E016E0001000C0A0EB8
:104F40000A01136F0D0E126F0A0E156F0F0E146FFC
:104F5000000177D70CCA13FA0BCA12FA0ECA15FA57
:104F60000DCA14FA10CA17FA0FCA16FA96DF01C052
:104F700011FA0A011151016E0001AAEF29F00A018C
:104F8000176B166B196B186B81B8FED781A8FED70B
:104F900081A804D0162BD8B4172BFAD781B804D027
:104FA000182BD8B4192BFAD71251E96E13CAEAFF9D
:104FB00017CAECFFED5216CAEFFF1451E96E15CA7D
:104FC000EAFF19CAECFFED5218CAEFFF000E016E9E
:104FD0000001F6EF27F00A0E0A01136F0D0E126F93
:104FE0000A0E156F0F0E146F0001C9D70CCA13FA01
:104FF0000BCA12FA0ECA15FA0DCA14FA10CA17FA19
:105000000FCA16FA4ADF01C011FA0A011151016EE6
:105010000001C9EF29F0000E016EE1EF29F00A014D
:10502000176B166B196B186B81BAFED781AAFED766
:1050300081AA04D0162BD8B4172BFAD781BA04D082
:10504000182BD8B4192BFAD71251E96E13CAEAFFFC
:1050500017CAECFFED5216CAEFFF1451E96E15CADC
:10506000EAFF19CAECFFED5218CAEFFF000E016EFD
:10507000000146EF28F00A0E0A01136F0D0E126FA1
:105080000A0E156F0F0E146F0001C9D70CCA13FA60
:105090000BCA12FA0ECA15FA0DCA14FA10CA17FA78
:1050A0000FCA16FAFADE01C011FA0A011151016E97
:1050B0000001E8EF29F00A010B6B0001D3DD01527A
:1050C00004E10A010B6B0001E1DD0A010B6B000139
:1050D000F1DDF5DD000E016E02EF2AF0C08EC28216
:1050E000C2B2FED70A01176B166B176BC4CF16FA44
:1050F00016CA17FA166BC3CF18FA1A6B1851006E3E
:105100001A51000B036E005016130350171316515B
:10511000016E1751026E000197EF28F013CA03F0D9
:105120000A011251146F13CA15FA0001D7D715CA14
:10513000EAFF14CAE9FF02C0ECFFED5201C0EFFF25
:10514000000E016EABEF28F00A0E0A01136F0D0E70
:10515000126F0001E3D701C011FAD8900A010D3592
:105160000F6F0E35106F0D510F270E5110230B517D
:10517000E96E0CCAEAFF10CAECFFED520FCAEFFF4E
:105180001151016E0A012AEF2AF08FDC000E016E28
:105190000AEF2AF010CA11FA700E0A011117113B1A
:1051A0000F0E1117126B010E006E1151016E04E00B
:1051B000D8900036012EFCD70050121310CA13FAF3
:1051C0000F0E1317196B12CA18FA010E125D006E3A
:1051D000000E1959036E00501A6F03C01BFA176AAC
:1051E000F2BE178EF29EC16B100EC06F03C0C3FAE1
:1051F0001ACAC2FA000186EC05F017BEF28E02C090
:1052000017FA01C016FA0A01196B12CA18FA036AD2
:1052100013511A6F03C01BFA176AF2BE178EF29E63
:1052200019CAC1FA12CAC0FA03C0C3FA1ACAC2FA2A
:10523000000186EC05F017BEF28E01500A0116251A
:10524000146F02501721156F1451016E1551026E23
:10525000000161EF29F02FDC720E0A010E6F0001D0
:105260007ADC015204E07CDC010E016E35D0430E85
:105270000A010E6F00016FDC015204E071DC020EC6
:10528000016E2AD06DDC17DC730E0A010E6F00016F
:1052900062DC015204E064DC030E016E1DD00A01E1
:1052A0000E6B0001A5DC01C00DFA5ADC0CCA03F03C
:1052B0000A010B510E6F0CCA0FFA0DCA10FA000149
:1052C00069D70FCAEAFF0ECAE9FF02C0ECFFED5230
:1052D00001C0EFFF000E016E11EF2AF00A01055127
:1052E000F70FD8B0B7D0090F00012DEF2AF057EC17
:1052F00025F00A0E0A010C6F060E0B6F00017DDC13
:1053000006CA0CFA04EC24F00A01A4D0DAD40A0E7E
:105310000A010C6F060E0B6F0001F3D406CA0CFADB
:1053200004EC24F00A0196D0FFDC0A0E0A010C6F8F
:10533000060E0B6F00011EDD06CA0CFA04EC24F009
:105340000A0188D07BDD0A0E0A010C6F090E0B6F73
:105350000001F5D50A0EE8CFEAFFE96EEFCF0BFAB0
:105360000BCA0CFA04EC24F00A0EE8CFEAFF090E8F
:10537000E96EEFCF0BFA0BCA0CFA04EC24F00A0129
:1053800069D05CDD0A0E0A010C6F090E0B6F00017B
:1053900022D60A0EE8CFEAFFE96EEFCF0BFA0BCA6E
:1053A0000CFA04EC24F00A0EE8CFEAFF090EE96ECD
:1053B000EFCF0BFA0BCA0CFA04EC24F00A014AD026
:1053C0002AD60A0E0A010C6F090E0B6F000153D684
:1053D0000A0EE8CFEAFFE96EEFCF0BFA0BCA0CFA20
:1053E00004EC24F00A0EE8CFEAFF090EE96EEFCFD5
:1053F0000BFA0BCA0CFA04EC24F00A012BD00A01B8
:1054000029D059D60A0E0A010C6F070E0B6F000146
:105410009BD6BBD60A0E0A010C6F070E0B6F00015C
:105420001AD70A0EE8CFEAFF080EE96EEFCF0BFAA3
:105430000BCA0CFA04EC24F00A0EE8CFEAFF070EC0
:10544000E96EEFCF0BFA0BCA0CFA04EC24F00A0158
:1054500001D00A01090126EF2EF0F2CF0EF0F29EE4
:10546000E8247F0FF66E540EF76ED8B0F72A0A00C4
:10547000F550FA6E0800F5500EBEF28EF96E125419
:1054800044538253C05328530C53EE52FE530254DC
:10549000176AF2BE178EF29E600E0A017F6F780EB9
:1054A000806F00015BEC0EF017BEF28E176AF2BE41
:1054B000178EF29E05CA7FFA95EC0EF017BEF28E9B
:1054C000176AF2BE178EF29E140E0A017F6F00015A
:1054D000C1EC0EF017BEF28EF0EF2DF025DC0A0EB7
:1054E0000A010C6F050E0B6F000144DC0A01055127
:1054F000016E0001F7EF2DF0176AF2BE178EF29ED3
:10550000D60E0A017F6FD00E806F00015BEC0EF0AB
:1055100017BEF28E176AF2BE178EF29E010E0A01B6
:105520007F6F000195EC0EF017BEF28E176AF2BE87
:10553000178EF29E05CA7FFA95EC0EF017BEF28E1A
:10554000176AF2BE178EF29E0A017F6B000195EC7E
:105550000EF017BEF28E0AEF2EF057EC25F00A0E71
:105560000A010C6F050E0B6F0001FDEC25F00A011E
:105570000551016E00010DEF2EF0176AF2BE178E75
:10558000F29E750E0A017F6FC80E806F00015BEC02
:105590000EF017BEF28E176AF2BE178EF29E05CA83
:1055A0007FFA95EC0EF017BEF28E176AF2BE178ED8
:1055B000F29E0A017F6B000195EC0EF017BEF28E91
:1055C00020EF2EF0176AF2BE178EF29E140E0A011B
:1055D0007F6F0001C1EC0EF017BEF28E23EF2EF0AC
:1055E000F86AD09E0D8EEA6AE96AC150C00B0F09B5
:1055F000C16E070EB46E8A8201019497DA6BDB6B81
:10560000949BFF6B400E0201006F016B500E026F06
:10561000036B600E046F056B700E066F076B040E54
:10562000086F0901EC6BED6BEE6BEF6BF06BF16BE0
:10563000F26BF36BF46BF56BF66BF76BF86B0001C9
:105640003AEF1CF0150EE8CF04FA080E0A01036FBA
:10565000030E056F04CA07FA03CA06FA000146ECF6
:105660001CF01A0EE8CF04FA300E0A01036F040E84
:10567000056F04CA07FA03CA06FA000146EC1CF0DB
:105680001D0EE8CF04FAD80E0A01036F050E056F50
:1056900004CA07FA03CA06FA000146EC1CF031EF0F
:1056A0001DF047EF1DF0C00EF2123DEF1FF0DCEFD2
:1056B0001FF0E9EF1FF0ECEF1FF0EEEF1FF0090114
:1056C000FB6BE86BE96BEA6BEB6B036AEB51E50F85
:1056D000E96E070E0320EA6EEF6A0001BDEF23F0CA
:1056E00001B003D00A01029302D00A010283010132
:1056F000949D94AD0FD00901FB6BE86B000152EC57
:1057000022F001B003D00A01029302D00A01028301
:105710000101949D0A0102B39ED2010194AD02D011
:105720000A0199D2010E0901FB25FC6F176AF2BE2E
:10573000178EF29E0A01C16BFBC9C0FAC36B030E40
:10574000C26F000186EC05F017BEF28E0150090F02
:105750000901F96F020E0220FA6FF951E96EFA5150
:10576000EA6EEF50DE0FD8B071D2220F00015DEF6C
:105770002EF0090E0A010B6FFF0E0A6F0001EBEC11
:1057800023F00901F951E96EFA51EA6EEF50000A6F
:10579000000103E0010A08E00AD00901FF1D0A0127
:1057A000006F002B000103D0FFC900FA00D000CA2F
:1057B0000CFA04EC24F0090149D2090E0A010B6F1E
:1057C000FE0E0A6F0001EBEC23F0090E0A010B6FCD
:1057D000FD0E0A6F0001EBEC23F00901F951E96EAF
:1057E000FA51EA6E020EEF5CFB0F3BE2050F00017F
:1057F0002EEF2EF00901FE51FD250A01006F09016F
:1058000030D00901FE51FD5D0A01006F090129D068
:105810000901FD51FE03F3500A01006F090121D077
:10582000176AF2BE178EF29EFDC9C3FAFEC9C4FA0A
:10583000EEEC0BF017BEF28E01C000FA090111D098
:10584000176AF2BE178EF29EFDC9C3FAFEC9C4FAEA
:10585000EEEC0BF017BEF28E00C000FA090101D089
:10586000090100CA0CFA000104EC24F00901EED190
:10587000090E0A010B6FFE0E0A6F0001EBEC23F01C
:10588000090E0A010B6FFD0E0A6F0001EBEC23F00D
:105890000901F951E96EFA51EA6E070EEF5CFA0F51
:1058A000D8B06AD0060F000145EF2EF00901FE5175
:1058B000FD5D02E0000E01D0010E016E01B003D0CB
:1058C0000A01029102D00A010281090155D00901A1
:1058D000FE51FD5D02E1000E01D0010E016E01B02E
:1058E00003D00A01029102D00A010281090144D0C9
:1058F0000901FE51FD5D02E3000E01D0010E016EB3
:1059000001B003D00A01029102D00A01028109010B
:1059100033D00901FD51FE5D02E2000E01D0010EFF
:10592000016E01B003D00A01029102D00A01028186
:10593000090122D00901FD51FE5D02E3000E01D0F4
:10594000010E016E01B003D00A01029102D00A01DA
:105950000281090111D00901FE51FD5D02E2000E34
:1059600001D0010E016E01B003D00A01029102D0F4
:105970000A010281090100D00A0102A103D0010E2F
:10598000006F01D0006B00CA0CFA000104EC24F097
:1059900009015CD1010E0901F925E96E000EFA2119
:1059A000EA6EEFCF05FA05CA0CFA000104EC24F008
:1059B00009014CD1010E0901F925E96E000EFA2109
:1059C000EA6E036AEF50E50FE96E070E0320EA6EF8
:1059D000EFCF06FA020EF925E96E000EFA21EA6E03
:1059E000EF500A010625036ABC0FE96E080E03207A
:1059F000EA6EEFCF08FA08CA0CFA000104EC24F0B2
:105A0000090124D1010E0901F925E96E000EFA21E0
:105A1000EA6E036AEF50E50FE96E070E0320EA6EA7
:105A2000EFCF06FA020EF925E96E000EFA21EA6EB2
:105A3000EF500A010625036ABC0F086F080E032009
:105A4000096F09CA0BFA08CA0AFA0001EBEC23F045
:105A50000901FCD0010E0901F925E96E000EFA21B9
:105A6000EA6E036AEF50F40FE96E070E0320EA6E48
:105A7000EF50FC6FEBD0090E0A010B6FFF0E0A6F9F
:105A80000001EBEC23F00901FF2D0FD0010EF925E9
:105A9000E96E000EFA21EA6E036AEF50F40FE96E28
:105AA000070E0320EA6EEF50FC6FD0D0090E0A01FA
:105AB0000B6FFF0E0A6F0001EBEC23F00901FF539F
:105AC0000FE1010EF925E96E000EFA21EA6E036A74
:105AD000EF50F40FE96E070E0320EA6EEF50FC6FF3
:105AE000B5D0FCC905FA11EF24F0010E0901F92522
:105AF000E96E000EFA21EA6E036AEF50F40FE96EC8
:105B0000070E0320EA6EEF50FC6FA0D0020E0901D1
:105B1000F925E96E000EFA21EA6E036AEF50580F7C
:105B2000E96E080E0320EA6EEF500A01016F010EC4
:105B30000901F925E96E000EFA21EA6EEFCF05FAA8
:105B400005CA06FA01CA07FA00011FEF24F081EF27
:105B500024F0090E0A01066FFC0E056F0001E4EF48
:105B600024F0090E0A01066FFF0E056F0001FEEF1B
:105B700024F0FFC90CFA04EC24F0090167D0090EE7
:105B80000A010B6FFF0E0A6F0001EBEC23F0FFC957
:105B900005FA00EF25F0090159D0090E0A010B6F33
:105BA000FF0E0A6F0001EBEC23F0FFC905FA26EFA8
:105BB00025F0090E0A010B6FFF0E0A6F0001EBECD6
:105BC00023F0FFC905FA6EEF29F0090E0A010B6FE9
:105BD000FF0E0A6F0001EBEC23F0FFC905FA58D461
:105BE000090134D00A010283090130D077D401C001
:105BF00000FA00CA0CFA04EC24F0090127D0090EBF
:105C00000A010B6FFF0E0A6F0001EBEC23F0FFC9D6
:105C100005FA72D409011AD0A0D401C000FA00CA52
:105C20000CFA04EC24F0090111D0090E0A010B6FE3
:105C3000FF0E0A6F0001EBEC23F0FFC905FA9DD4BB
:105C4000090104D0BFD4090101D00901FCC9FBF945
:105C5000010160D50A0101014CD50300F2CF0EF01D
:105C6000F29EE824810FF66E5C0EF76ED8B0F72A2C
:105C70000A00F550FA6E0800F5500EBEF28EF96E6D
:105C8000F4570258105820584058F2CF0EF0F29EA8
:105C9000E824AF0FF66E5C0EF76ED8B0F72A0A0054
:105CA000F550FA6E0800F5500EBEF28EF96EAC5843
:105CB000CE58F058125934595659F2CF0EF0F29E80
:105CC000E824DF0FF66E5C0EF76ED8B0F72A0A00F4
:105CD000F550FA6E0800F5500EBEF28EF96E72574E
:105CE0007257BA57BA57BA57BA57BA577058705806
:105CF00070587058705870589459B459045A545A7E
:105D0000765AAC5AE25A0C5B4E5B525B7E5B625B2E
:105D10009A5BE45BB25BCA5BEC5BFE5B185C2A5C83
:025D2000445CE1
:10B98000080E016E000000008C9695960000B837F6
:10B99000839CD8B0958CD8A0959C958683A6CEEF35
:10B9A0005CF0012EC2EF5CF000008C9695960000D2
:10B9B000958C00000000958683A6DCEF5CF0016AA0
:10B9C000000083BC01808C969596839C959C000C0E
:10B9D000958C000095860000839C959C00008C96B9
:10B9E0009596A00EB86FC0EC5CF0036AB50EE96ED8
:10B9F00003C0EAFFEFCFB6F0B6C0B8F0C0EC5CF021
:10BA0000036AB40EE96E03C0EAFFEFCFB6F0B6C02A
:10BA1000B8F0C0EC5CF0958C000095860000839C2B
:10BA2000959C00008C969596000C080EBB6F00C08C
:10BA3000BCF0958C0000958683A61CEF5DF083BC5E
:10BA4000D88083ACD8900136000095968C96BB2F99
:10BA500019EF5DF0958C0000839CBC51D8A4959C97
:10BA60000000958683A632EF5DF000008C969596D7
:10BA70000000839C959C000CF250036EF29EA69CE5
:10BA8000A68EA6840F01550EA76EAA0EA76EA682DB
:10BA900000000350F2120001000C958C0000958606
:10BAA0000000839C959C00008C969596A10EB86F23
:10BAB000C0EC5CF0B76B010EB65DB75DD8B070EF4F
:10BAC0005DF0B751B425E96E000EB521EA6E010EA6
:10BAD000006E15EC5DF00150EF6EB72B5BEF5DF083
:10BAE000B751B425E96E000EB521EA6E006A15EC77
:10BAF0005DF00150EF6E959C0000958683A67EEF69
:10BB00005DF00000000000000000958C0000000CBB
:10BB1000F86AB5C0F7FFB4C0F6FFB7C0EAFFB6C019
:10BB2000E9FFB8C000F00900F5CFEEFF002E93EF5B
:10BB30005DF0F86A000CD08CF86AB5C0F7FFB4C0AD
:10BB4000F6FFF650070B006EF80EF6160A00B7C0A7
:10BB5000EAFFB6C0E9FFB8C002F002C001F0005031
:10BB6000022602040709026E022AF6500066C3EF9D
:10BB70005DF0010F3F0BD8A4C3EF5DF0A68809006C
:10BB80003CEC5DF00A000066D0EF5DF0EECFF5FF13
:10BB90000152D8B4D1EF5DF00F000106D3EF5DF094
:10BBA00000060B000C00070EF614070AD8A4DBEF02
:10BBB0005DF03CEC5DF0022EB5EF5DF0F86A000C34
:10BBC000B7C003F0B651E96E03C0EAFFEF50BA6F99
:10BBD000B9C003F0B851E96E03C0EAFFEF50BB6F84
:10BBE000BBC0BCF0BAC0BBF0BCC0BAF0B551BB1B07
:10BBF000BB39006E0F0E00160050BB1BBB39006E28
:10BC0000F00E00160050BA1BBB31006E003200323D
:10BC10001F0E00160050BA1BBB39006EF00E001646
:10BC20000050D89000360050BB1BB7C003F0B6518F
:10BC3000E96E03C0EAFFBAC0EFFFB9C003F0B85124
:10BC4000E96E03C0EAFFBBC0EFFF000CFFFFFFFF80
:10BD0000F86AD09EEA6AE96A0F0EC16E070EB46E39
:10BD10008B84979C8E8C8C8EB16BB06BAD6B050E4B
:10BD2000AC6FAB6B400EAA6FC00EB36FB26BB56B4E
:10BD3000B46BE8EC5CF0A10EB86FC0EC5CF0010EE7
:10BD4000006E15EC5DF001C008F0010E006E15EC00
:10BD50005DF001C009F0036AB10EE96E03C0EAFFAD
:10BD6000010E006E15EC5DF00150EF6E036AB00E2F
:10BD7000E96E03C0EAFF010E006E15EC5DF00150A4
:10BD8000EF6E006A15EC5DF001C006F0A76BA66BC4
:10BD90000B6A0C6A076A0650075CD8B0AFEF5FF019
:10BDA000ADC0B5F0ACC0B4F0E8EC5CF0A10EB86F7B
:10BDB000C0EC5CF0036AA10EE96E03C0EAFF010E5D
:10BDC000006E15EC5DF00150EF6E036AA00EE96E97
:10BDD00003C0EAFF010E006E15EC5DF00150EF6E3E
:10BDE000036AA90EE96E03C0EAFF010E006E15ECAE
:10BDF0005DF00150EF6E036AA80EE96E03C0EAFF22
:10BE0000006A15EC5DF00150EF6EA051C00BA26FFF
:10BE1000A151A36FA0513F0BA46FA151000BA56FBF
:10BE2000A651A25DD8A41AEF5FF0A751A35DD8B4C4
:10BE30002CEF5FF0A453D8A422EF5FF0A553D8B441
:10BE40002CEF5FF0D08CF86AA3C0F7FFA2C0F6FF1A
:10BE5000A6883CEC5DF0F86AA3C0A7F0A2C0A6F0EB
:10BE6000040EAC27000EAD23ABC0B5F0AAC0B4F0F1
:10BE7000E8EC5CF0AF6BAE6BAF51A95DD8A0ACEF56
:10BE80005FF0D8A449EF5FF0A851AE5DD8B0ACEF39
:10BE90005FF0AF510708D8A063EF5FF0D8A456EF6A
:10BEA0005FF0AE519308D8A063EF5FF0B56B100E52
:10BEB000B46F100EB66F4DEC5DF0100EAA27000E99
:10BEC000AB2372EF5FF0B3C0B5F0B2C0B4F0B76BA4
:10BED000100EB66F100EB86F88EC5DF0100EB22722
:10BEE000000EB323A1C0B5F0A0C0B4F0B76B100E24
:10BEF000B66F100EB86F9BEC5DF0A1C0B5F0A0C09E
:10BF0000B4F0B76B100EB66F100EB86F88EC5DF022
:10BF10000E6A0E500F08D8A0A3EF5FF0100E0E248B
:10BF2000E96EEA6AD8B0EA2AEFCFB4F0B4C0B5F04F
:10BF3000B76B0B0EB66FB96B0C0EB86FE0EC5DF023
:10BF40000E2A89EF5FF0100EA027000EA123AE2B62
:10BF5000D8B4AF2B3CEF5FF0072ACBEF5EF008C000
:10BF6000B5F0B76B0B0EB66FB96B0C0EB86FE0EC9B
:10BF70005DF009C0B5F0B76B0B0EB66FB96B0C0E68
:10BF8000B86FE0EC5DF0AB6B400EAA6FAD6B050EC9
:10BF9000AC6F0B52D8B4D1EF5FF00C52D8A48CEF39
:10BFA0005EF08C9E8B94979C8E9CFF000300FFFF9D
:020000040030CA
:0E00000000220C0E83018100FFC0FFE0FF40D4
:00000001FF
